:020000041102E7
:1000000070B501F079F840201F4C0223FE211F4AF1
:10001000207401F0D1F8002821D10223FF211C4ACD
:10002000207C01F0C9F8051E19D19022022112028C
:10003000207C01F03BF9032007F032FF80220221EF
:100040005201207C01F032F92900207C01F00EF9E8
:1000500023681049002B12D001F09CF870BDCC220F
:100060003820AC219201207401F020F9002802D040
:1000700000232374F0E72368002BEDD106490C22FE
:10008000200007F025FDE7E78864FF1F9464FF1F49
:100090009664FF1F588102114C810211F7B5164B6F
:1000A0000192C318021D0020009388235B05D3181A
:1000B0001B685C1C1AD09CB2402C18D88D781E0C82
:1000C000AC466746CD782D023D43AE4206D101983D
:1000D00000280ED110000C70240A4C7003249BB22F
:1000E0000733A343D218009B9A42DED3FEBD4432AD
:1000F000F9E71000FAE7C046FC0F0000802213B5B4
:1001000003000324019189B2520107319B18A143D6
:1001100004305A1A88235B05C3181B68591C03D185
:1001200090429241104016BD99B2402907D80B0069
:100130000733A343C0189042ECD30020F3E74430C8
:10014000F9E7134B134A1B68126810B5FA2493425F
:1001500001D81A00F824104BE4021B689A4210D808
:1001600013000E4A12689A420ED3013307D1F823C6
:10017000DB029C4203D10A49054807F0A1FD20009B
:1001800010BDFC24E402ECE7FE24E402F7E7C046DD
:1001900000C0071100D0071100E0071100F007119F
:1001A000FFFFFF7FF0B59BB0150004900391402A3C
:1001B00000D9A0E006AB59801A80FFF7C2FF040007
:1001C000042816D9002206A9FFF768FF052810D9D0
:1001D00006AB1B88AB420CD1002D07D0514B2A0037
:1001E0000499C01807F034FD002802D101201BB08B
:1001F000F0BD06AB1D8020000699FFF77FFF041EAF
:100200007BD1069B0793FFF79CFF80235B01C618F9
:10021000802307001B039E4201D3F826F6028823A1
:100220005B05F31801931B68013302D0019807F0B6
:100230001FFD3D49019807F043FD3B1D0293331D0F
:1002400005938822029B52059B181B6808935A1C31
:100250003CD044219AB20091402A04D80320D11DF9
:10026000814389B2009103991B0C8B4224D0402A10
:1002700022D80122300008A9FFF710FF021E1BD16F
:10028000380008A9FFF70AFF0400042831D9009AB2
:10029000059B9B1880225201B218934240D28823BA
:1002A0005B05C118009A09A807F0EAFC1D4B009AEB
:1002B00009A9F01807F0ACFB009A029B944663442E
:1002C00002931A4B029AFB189A42BAD388235B0511
:1002D000FC1821680198013907F0F2FC200007F0B2
:1002E000C7FC039A07AB5A8030000799FFF706FF57
:1002F0000400002C03D1002079E70428FBD98823CF
:100300005B05E018069907F0DBFC0323EA1C9A431F
:1003100000D16BE7034B0499E01807F079FB65E720
:100320000424ECE704000011FFFFFF7FF80F00003A
:10033000F7B505001400402A21D8002701AE7180CE
:100340003780FFF7FEFE042816D93A003100FFF788
:10035000A5FE042810D93688BC420BD0BD4209D076
:10036000221CB44200D9321C064B92B2C11828009C
:1003700007F086FC30B2FEBDC04300B2FBE70320AD
:100380004042F8E70400001137B5042204000D00D4
:1003900001A81649FFF7CCFF020004280BD1019BEE
:1003A000A34208D3AB4204D0104901A80195FFF73E
:1003B000F9FE01203EBD0E4C23682000019307F09A
:1003C00057FC019920000139019107F079FC802345
:1003D0005B01E418074B9C42EED10422034901A8BB
:1003E0000195FFF7DFFE0020E4E7C0465555000009
:1003F00000C0071100000811F7B50F490F4B0A683C
:1004000004001A4084235B0013430B60030003279E
:100410001033019300252E00112007F049FB084BF3
:100420001B683B40AB4002351E43202DF4D1019B9D
:1004300040C4A342EED1F7BD5CF0004000FEFEFFD9
:1004400064F00040802270B5B04CB14BD200002166
:1004500020001C6007F0D4FC2300AE4A88331A60E9
:10046000AD4B1A786E23002A00D01133E3620A23C1
:100470002365AA4B1878AA4BA0630138E361C3B285
:10048000032B01D810232362A64B37226361C823B4
:10049000DB00A36123008C331A60082336210F3A56
:1004A000E518E16323646264E9670439251DE9679F
:1004B00025003B26BC352E602500C0352B6025006D
:1004C000C4352A6025000636CC352E602500083E4E
:1004D000C8352E602500D03529602100D4310B604D
:1004E0002100D8310A6021000225E0310D6025008D
:1004F0004221DC35296025001B3EE4352E602500B5
:10050000E8352B602500EC352A6022000525F43201
:1005100015602200F0321160220018319032116013
:1005200022009432136023003C2298331A60AF23D8
:10053000DB0023607C4B2363032805D807F088FD8C
:10054000330235371523636096232100FA225B00BE
:10055000A360E360C8332361744BFC319200A36451
:100560000A606262724A734DA2627322E2656D3A5A
:100570006265A2650232E5644A60022161669621E5
:100580008900A166626709210022E166A2676A49C3
:100590006A4A6B4E2167E2673560032811D807F07D
:1005A00057FD9C08A4AC1023CDE70E23CBE70C230A
:1005B000C9E720001A259C30056020000735A030CF
:1005C00005602000A83003602300FA20F833800083
:1005D000186023006420A433186023005F38AC3314
:1005E000186023000338B03318602300C630B433DA
:1005F000186023000020B833186023003825FC332E
:100600009D60504D5A665D644F4D9A64DD6196253C
:10061000AD001D624D4D9A675D62F53DFF3D9D62E7
:100620001E254B4ADD6618675867D9651966DA6773
:10063000BE23C021474A5B00E250474B490063504C
:1006400004316250C4225200A350FA23E4205B001C
:100650000432A3500432A3504049414A414BD16077
:100660004149800019504149E938FF381950404943
:10067000043019503F491038D1613F4911633F4957
:1006800051633F4911603F49195019003E48F83104
:1006900008603E49D16586213D4A89005A503D4A4D
:1006A00010395A503C4A0C315A501A003B49083212
:1006B000D1671A003A49B43211608821394A890059
:1006C0005A501A00384988321160384ADA6407F003
:1006D0004FFC012007F054FA70BD200014259C3017
:1006E000056020000435A0306AE7200010259C300A
:1006F000056020000335A03062E720000E259C3005
:10070000056020000235A0305AE7C0460004FF1FF4
:100710004467FF1F3072FF1F2447FF1F4A0AFF1F55
:100720003A07000080C3C9019A02000050C30000CC
:100730006A180000280A0000204E000088130000FC
:10074000F009FF1F0040001168100000C4090000FC
:10075000DC05000040420F0010270000FD1BFF1FBA
:10076000FC00FF1F0000FF1FED30FF1F1534FF1FAF
:10077000AD32FF1FD91FFF1FF51FFF1FA121FF1F54
:10078000491FFF1F8D2AFF1F552EFF1FD918FF1F5E
:10079000D127FF1F9929FF1F8528FF1F3925FF1F1C
:1007A0004525FF1F491EFF1F011FFF1FC11DFF1F02
:1007B000F7B50B0CFF270122009300233C001E001D
:1007C0001D009446019089B262469A40100008408C
:1007D00018413618B6B2FF2F02D1012E00D19FB2B8
:1007E000009802401A41AD18ADB2FF2C02D1012D84
:1007F00000D19CB20133102BE6D10320012E07D18A
:10080000012D04D1019B2401E4191C700138FEBDA7
:10081000102EFCD10238102DF9D00230F7E710B5B8
:10082000064C2378002B07D10548FFF7E5FD054866
:10083000FFF7E2FD0123237010BDC0460467FF1FD0
:100840001867FF1F0867FF1FF0B58BB00D0001236D
:100850000190102936D8FFF7E2FF00231A001B4849
:10086000C15C01335218102BFAD1023B002A29D067
:10087000174B184C1F68002306A9E25C1600FA5CAF
:1008800056405E540133102BF7D102AA07F0D8F876
:100890002A0002A9019807F01BF907F0F9FA23686A
:1008A0001B18236007F0F4FA63681B18636007F0F5
:1008B000EFFAA3681B18A36007F0EAFAE3681B18B5
:1008C000E360002318000BB0F0BDC0461867FF1F9F
:1008D000C445FF1F0867FF1FF0B502230124504ED7
:1008E000504D8FB0002033702C7006F0E5F807F003
:1008F000EFFAFFF7A7FD07F0B3FB1F2200214A4BD9
:100900000EAF1A70494B1C70494B1970494B19684E
:100910009143163A0A431A60602219689143403A9B
:100920000A431A6007F0BCF907F04AF9C120FF2119
:10093000414B80001A588A431A50C5229200985899
:100940008843BF390143995098583C490840802159
:10095000C9010143802099509958C0050902090A2C
:100960000143995080213648490107F029FA0323B1
:100970002200344901940093334807F059FB2C229C
:10098000324903A807F07CF903AC6178207802347F
:1009900005F020FEA742F8D10121002005F004FF58
:1009A0000121002005F030FF0121092005F02CFF76
:1009B000274B284A196803201140A022D2020A437B
:1009C0001A608022196892040A431A601968224A40
:1009D0001140802292030A431A60204B204A93421E
:1009E00000D8012007F0E4F807F03AFA07F0F0FA2F
:1009F000307807F09DF82878C0B207F0A9FA07F020
:100A00000FF91849042007F033F806F021F800F038
:100A10009DF800F033FD00F009FA00200FB0F0BDA2
:100A20004A0AFF1F2447FF1F480AFF1F490AFF1FEA
:100A3000680AFF1FBCF0004000E100E0FF00FFFF7C
:100A40002847FF1FAC59FF1F2857FF1F7080021156
:100A500014F00040FF7FF8FFFFFF9FFF3072FF1F81
:100A60000080FF1F3B00010870B500252849294A76
:100A700029484D6308CA1B051B0DED188242F9D1A8
:100A80000022264B8B63264B08211A628022254BBD
:100A90009205DA67244BDA688A43DA60234A1278CF
:100AA000012A03D09A6822490A409A600121EE2463
:100AB0002048E40002686C438A430260DA6811202F
:100AC0008A43DA6007F054F9112007F061F8112029
:100AD00007F016FA184A200C0400642390420AD842
:100AE000FA220023D200904205D9144B0A21C018E3
:100AF00007F046F9C3B2124A1372124BD4801B7826
:100B0000002B04D1104B1021187807F071F970BD3B
:100B1000000005408805054000060540FF01000073
:100B200000F0004004E100E03CF000404A0AFF1FF2
:100B3000FFDFFFFF00380040B70B000030F8FFFF79
:100B40009C64FF1FBE66FF1FB464FF1F002210B528
:100B50001100112007F024F810BD0000F8B50023A3
:100B600001250826394F3A4C3B62E3681120AB431C
:100B7000E360E368B343E36007F00AF8112007F08D
:100B8000F7F8112007F00CFA4023226829001343DC
:100B9000236080236268DB02134380226360A368C2
:100BA00007201343A360A3682A4A1340A36080234D
:100BB000A2689B0113431022A360236C9343236418
:100BC000236C2B43236480235B003B62226B224B0C
:100BD0001A402263626B1A406263A26B1A40A263DE
:100BE000E26B1340E3631D4AE3681340E36005F0E2
:100BF000DBFD2900072005F007FE8021184A11209F
:100C0000536C0B43536407F0EBF9FD21154B164A67
:100C100089005A508023C720626B5B0313436363D0
:100C2000E36880003343E360E368104A1D43104BE0
:100C3000E56019581140802212020A431A5080229E
:100C400092051A600B4B5E63F8BDC04600F0004091
:100C50003CF00040FFFFDFFFEFFFEFFFFFFF7FFFF4
:100C6000003800400000FF1F690A0211FF00FFFF6B
:100C700000E100E00000054030B503A804880B2027
:100C8000002C0ED14968074D0878497809020143C4
:100C90000A20A94205D1012120001980024B1B7AAC
:100CA000137030BD192A00009C64FF1FF7B51500B2
:100CB00008AA16884A680F4F147852781202224305
:100CC0000A24BA4214D10122DBB2019200962A0012
:100CD00006F00EFE041E0BD1074B1B68002B07D03D
:100CE00068782A7800021043424250410130984708
:100CF0002000FEBD022900002C64FF1F30B5012535
:100D000003790400BFB02B4212D00A49408806F094
:100D10005BF928420CD06A46074B69465B8D5580CB
:100D20001380064B60881B7A1371002203F00EFAC1
:100D30003FB030BD2464FF1F9043FF1F9C64FF1F22
:100D400010B50549054806F0F5F80421044A0548A0
:100D500006F0B2F810BDC0462464FF1FFFFF00007C
:100D60009C8002119043FF1F10B5024804F074F8F4
:100D700010BDC046FD0C02110623837010330371B1
:100D8000443B43712A3383714433C37100230222ED
:100D9000012110B503720E4B027041701C888172E4
:100DA0004472197A0273C1729A784273DA78827344
:100DB0000322C2731A7902745A7942740C22827423
:100DC0009A79C274DB7903751123C37010BDC046D4
:100DD0009C64FF1F10B5142006F08AFF124B1422EA
:100DE0000021186006F014FF002006F079FE0120B3
:100DF00006F01EFF022006F04BFF032003F0D0FA9E
:100E0000042005F0E5FA052002F01EFD062003F09F
:100E1000DBF9072000F00AFF082006F02DF8092072
:100E200000F014FD10BDC0463064FF1F10B506F081
:100E30003FFF012006F0FCFF07F0BAF8002010BDCC
:100E400070B50D7A100004AA2C00168810221440E8
:100E5000154220D1002E20D10A78022A18D14A68E2
:100E6000557816780E4A2D023543954205D00D4A25
:100E7000954209D01C800A2404E01422C9681A8013
:100E800006F026FE200070BD0C2207491A80F7E705
:100E90001C800124F6E70824F4E70B24F2E7C0469F
:100EA000F3FF0000F4FF0000A864FF1FF7B50E0079
:100EB000377A1D0008AB11003C001A8820231C4023
:100EC0001F4236D13378022B35D173681F785B7897
:100ED0001B023B431B4FBB4208D01B4FBB420ED0F3
:100EE0001A4CA3421BD00A242000FEBD002A24D1A4
:100EF000142D24D82A00F06806F0EAFDF4E7002A51
:100F00001BD1202D1BD82A00F06806F0E1FD104B04
:100F100004211D700F4B187806F06AFFE4E70124E6
:100F2000009201940A00EBB2310006F0E1FC0400EB
:100F3000DAE70824D8E70124D6E70B24D4E70D2408
:100F4000D2E7C046F3FF0000F4FF000002290000D2
:100F50003464FF1FB464FF1F094B10B504009842AE
:100F600005D0012904D12000064905F0E3FF10BD9A
:100F70000229FCD1013903F02DFF0028F3D0F6E758
:100F8000FEFF00005664FF1F10B504000749084823
:100F900005F0D0FF074803F09FFE0020E40704D5CA
:100FA0000621054A054805F087FF10BD5664FF1F5E
:100FB000FFFF0000590F0211E0800211D443FF1F10
:100FC00000B5BFB06A460B4B0B491B8801A81380C4
:100FD0000A4B1A7800F086FA6B4680B258800028D7
:100FE00005D0074B00226946188803F0AFF83FB0E0
:100FF00000BDC0461E44FF1F3564FF1F3464FF1F41
:101000002045FF1F70B5160004AA148805AA15789C
:101010004A685078117800022A4A08438018052847
:101020004BD807F015F803131E29343F0720042C72
:101030000BD80522121BAA4200D92A0022491A8085
:101040003000091906F044FD002070BD0720132C64
:10105000FBD81422121BAA4200D92A001B491A806D
:10106000EEE707200E2CF0D80F22121BAA4200D95F
:101070002A0017491A80E3E70720032CE5D8042249
:10108000121BAA4200D92A0012491A80D8E7072069
:10109000032CDAD80422121BAA4200D92A000E49D6
:1010A0001A80CDE70720032CCFD80422121BAA42B6
:1010B00000D92A0009491A80C2E700220A201A80B2
:1010C000C3E7C046DCD5FFFF2B8102117264FF1F0E
:1010D0001B81021116810211118102110C81021172
:1010E00010B50D21024A034805F0E6FE10BDC046CA
:1010F000008102113444FF1F10B50021162005F0B5
:10110000BFFB0121152005F0BBFB06F079FD0400B3
:10111000092006F045FF0022184BDA6661321A609A
:1011200019685B3A9143023A0A431A60144A94429E
:1011300009D10A22DA6107321A6200221A639A631D
:101140000132DA6310BD0F4A944203D11E22DA61E4
:101150000532F1E70C4A944203D13022DA610632BB
:10116000EAE70A4A944203D14322DA610832E3E70C
:10117000074A9442E1D16922F7E7C0460050004097
:101180000024F4000048E801006CDC020090D00369
:1011900000D8B80510B50024064B0920DC6606F01F
:1011A000F7FC2100162005F0FFFA2100152005F0BC
:1011B000FBFA10BD00500040F8B51C000023134D91
:1011C0000F00EB666860160006F02AFC01238022FF
:1011D000EB6623002F615200013B08D206F0F8FDB8
:1011E00008200B4A1168002C03D12000F8BD2A61A9
:1011F000F2E72B6F034203D02B69013C33700136B9
:1012000013685B1A012BEED90124EEE70050004071
:101210006008FF1F002370B5124D1400EB66686074
:101220000E0006F0FDFB01238022EB662300520036
:10123000013B08D206F0CCFD08200B4A1168002CB7
:1012400003D1200070BD2A61F2E72B6F034203D067
:101250002B69013C3370013613685B1A012BEED900
:101260000124EEE7005000406008FF1F002370B526
:101270000C4C0D00E366606006F0D2FB0123E366D0
:10128000256106F0A5FD8020074A80001168636B88
:10129000034205D113685B1A012BF8D9012070BDF8
:1012A0000020FCE7005000406008FF1F002370B5DD
:1012B000134C0E00E3666060150006F0B1FB0123DD
:1012C000E36626610F33626B1A42FCD02B0A23615E
:1012D0001023626B1A42FCD0EDB2256106F078FD56
:1012E0008020084A80001168636B034205D11368AF
:1012F0005B1A012BF8D9012070BD0020FCE7C04625
:10130000005000406008FF1F13B5344C237C002BB5
:101310005FD0FFF7F1FE207C38283FD107226946D5
:10132000FFF778FF002854D16B461B787F2B50D8ED
:10133000CC22AC219201207CFFF7B8FFFFF72AFFF7
:101340006B46D878F02302041B031A406B469B8837
:1013500023495BBA9BB21A4323680009534322898D
:101360001B0C9B184B806B465A789B7812031B0111
:101370001A4302436368534362891B0C9B181BB2D8
:101380008B80002B04DA0022154B9A80002016BDBA
:10139000144A9342FADD124B124AF6E769460422D8
:1013A000FFF738FF011E14D1207CFFF75FFFFFF726
:1013B000F1FE6B461A88236852BA92B253432289CF
:1013C00007491B0C9B184B806B465A8852BA92B245
:1013D000D0E7FEF715FE0120D9E7C0468864FF1F5D
:1013E0009C64FF1F0F27000010B51B4B1A793F2A82
:1013F00001D93F221A711979184A19481170182217
:101400001849028018480A8002804A809A79174851
:10141000802402800C208A80013242432401101C67
:10142000A24200D9201C124AC88010805A79002A92
:1014300001D101325A711A7A002A01D101321A728D
:101440005A791B7A0B4853430A21584306F098FCFB
:10145000094C206010BDC046A864FF1F480AFF1F4A
:101460001E45FF1FD046FF1F1C45FF1F1A45FF1FCB
:101470001845FF1F71020000B864FF1F10B5062158
:101480000020FEF781FF124C002807D10C2220001B
:10149000104906F01DFBFFF7A7FF10BD0C2220002E
:1014A0000D49FEF745FF0C2804D00C222000094905
:1014B00006F00EFB094C0C2220000949FEF738FF0C
:1014C0000C28E8D00C220021200006F0A1FBE2E766
:1014D000A864FF1F64810211FC0C00008864FF1FD8
:1014E000F50C0000F7B5040000200D000100824259
:1014F0000AD02B7860702370834206D11423638056
:101500000E3BA06063600C30FEBD552B19D1013A33
:10151000624E0C2A13D8002A0AD0691C300006F04B
:10152000D7FAFFF761FF0C2230005D49FEF73AFE63
:101530000C223100601C06F0CBFA0D20E4E70C22EF
:10154000EBE7562B10D1554D0C225649280006F0DA
:10155000BFFAFFF749FF0C2251492800FEF722FE8F
:101560000C222900601CE6E7252B17D1013A4E4ECC
:101570000C2A11D8002A08D0691C300006F0A8FAFD
:101580000C2230004949FEF70DFE11223100601C8B
:1015900006F09EFA1220B7E70C22EDE7262B0AD1BF
:1015A000414D1422280006F033FBFEF729FD1122DD
:1015B0002900601CECE7DC2B1DD1022A6BD96B786B
:1015C0006370AB78A3706E781B021E43032A05D0AC
:1015D000033A310092B2E81CFEF7E4FD102231001C
:1015E000E01CFEF7A5FE03000330002B00DB8BE7B9
:1015F0000220637088E7DB2B20D1042A4BD9A9781D
:101600006B7809021943EB782F791B040B433F06D3
:1016100010261F43052A05D0561F32003800691DC9
:1016200006F056FA05222900200006F051FA320091
:101630003900601D06F04CFA701D65E7DA2B2AD1DF
:10164000042A28D9AB7869781B020B43E97809048E
:1016500019432B791B060B43082A19D9AA796979F2
:1016600012020A43E979090411432A7A12060A434D
:1016700001921A601B68052229002000019306F0E0
:1016800027FA0422601D01A906F022FA09203BE78F
:10169000FE226270EEE7FF23AAE7C046A864FF1FA0
:1016A000FC0C0000648102118864FF1FF50C00002F
:1016B00070470000013870B5042809D806F0C8FC4E
:1016C000030921081200144B0221187806F090FB40
:1016D00070BD114B0821187806F0D2FB00220F4B89
:1016E0001A71F5E700240D4B0B4D082128781A6874
:1016F0001C719C7106F0CCF92100287806F0B0F935
:10170000E6E70123054C0821A371034B187806F086
:10171000B7FB00232371DBE7B464FF1FB864FF1F2E
:1017200010B5002903D10920013105F06DF810BD75
:1017300010B5084B084C9881D881188258822078BF
:1017400001F020FF0422054B012120781A7006F0D9
:101750004FFB10BDCE45FF1FEE66FF1FED66FF1F5E
:1017600010B501290DD11322064B002109209A71D1
:1017700005F04AF8044B1B78002B02D00348FFF712
:10178000D7FF10BDB864FF1FBE66FF1FC40900006D
:101790000300F0B50A4D8E18B14202D152008018F4
:1017A000F0BD0C782F6824093C5D0F271C700C7865
:1017B00001313C402F683C5D5C700233ECE7C04671
:1017C0001445FF1F10B50A4A0A49082005F01EF902
:1017D000092005F005F90121092005F015F8002080
:1017E00005F0FEF80121002005F00EF810BDC046FE
:1017F000211702116117021110B5114B1A781870D8
:10180000002A0ED000280BD10E4B1A78062A07D8D2
:101810005423D340DB0703D50B4B187801F0B2FEFD
:1018200010BD0028FCD0074B1B78012B02D0033BD6
:10183000022BF5D8044B0121187806F0D9FAEFE70E
:10184000BE66FF1FED66FF1FEE66FF1FF0B5554D2C
:1018500085B02870FFF7B6FFFEF7D2FB06F0E0FA7E
:10186000002002A90290039006F0FAF903224E49E3
:101870004E48FFF78DFF2D24030004221C704C49B5
:101880000130FFF785FF0222047002A90130FFF743
:101890007FFF0222474B484CDA87200006F0A0F970
:1018A000022815D0062220004449FEF741FD0628F3
:1018B0000ED00321200006F0F3F88D23E3706E3B79
:1018C00023710622193320003C496371FEF76AFC3C
:1018D0000E233B4F3B4C3C4E3B70013B237005229B
:1018E000043B300039496370019606F0F1F82D236E
:1018F000012237493748E371FFF74AFF0122364991
:10190000FFF746FF01222C49FFF742FF0020FFF7B7
:1019100073FF324E324A0121324B1278307801F097
:10192000F3FD3A78012723000021307801F0ECFD27
:1019300021782D4B0139019AC9B200201F7005F0A2
:10194000D9F9FA221B4B52019A81DA811A825A8202
:101950002021287806F094F80120404205F016FA7C
:101960000120404205F0B2FAFFF7BAFBFFF7E8F9B1
:1019700000F06EFC01204042FFF706FB380006F045
:10198000A7F9F72000F07CFF3900287806F030FA3C
:10199000287801F053FF154806F0FAFAFFF7DEF851
:1019A00005B0F0BDB464FF1F4446FF1F7264FF1F03
:1019B0009464FF1FCE45FF1F6509FF1FADAC0000FB
:1019C000BA66FF1F9B66FF1F9D66FF1F2B810211DA
:1019D0006709FF1FA366FF1F6609FF1FEE66FF1F53
:1019E0004845FF1F2945FF1F8C66FF1FC064FF1F6E
:1019F000F8B50A0020230D001A40194232D0414B9D
:101A00001B78002B2BD0404C404E23790133DBB2A6
:101A10002371327A9A4215D800272771FFF774FC98
:101A200063790133DBB26371727A9A4202D86771CB
:101A3000FFF794F8364F3800FFF79EF9390015206C
:101A400006F06EFAA379002B09D0013BDBB2A3713B
:101A5000002B04D1707964335843FFF769FE2020CE
:101A60006840F8BD0BB2002B0ADA2A4B187806F052
:101A700027F8002801D005F0DBFF80200002EFE707
:101A800002240E002640214206D01F4B01201A716D
:101A9000FFF7B2FE2000E3E70B0711D5FFF734FC98
:101AA00000F0F0FB184A194953790133DBB2537146
:101AB000497A994202D85671FFF750F80820CFE7CB
:101AC00010240E002640214206D00E4B1B78002B1E
:101AD000E0D1FFF749F9DDE70124214209D00E48A2
:101AE00000F068F806F09CFA3100092004F08CFE42
:101AF000D0E70424080020402142B2D0FFF760FA6A
:101B0000C8E7C046BE66FF1FB864FF1FA864FF1F7A
:101B10002945FF1FB464FF1F0C45FF1FF0B51B4B89
:101B20001B4F1B883A8804001A4E1B4D85B09A4201
:101B30000DD832889A420AD3184B1A882B889A42B9
:101B400005D1174A174B12881B889A421BD00520D3
:101B500000F0ECFE3B8802AA13803388019053808A
:101B60002B88114D93800F4B02A91B88D3800F4BFC
:101B70002A78188802F0F8FB0D4B08212878019A82
:101B80001C7006F0BDF805B0F0BDC0468A66FF1FA8
:101B90001E45FF1F1C45FF1F1A45FF1F8866FF1FBC
:101BA0008666FF1F1845FF1FEE66FF1F2045FF1FBB
:101BB0008466FF1F13B50C4B1C78002C11D1002834
:101BC00001D00A4B18600A4A0A4B11780A4A107869
:101BD0000A4A01920A4A0092002204F083FF200080
:101BE00016BD1124FBE7C046ED66FF1F8066FF1F90
:101BF000EC66FF1FDC66FF1FEE66FF1FC866FF1F57
:101C0000CC66FF1F10B5064B12201B78052B06D1A2
:101C1000044B13221988044B187801F063F810BDA7
:101C2000ED66FF1F2045FF1FEE66FF1F10B5002465
:101C30000122114B52421870104B1C70104B1A802D
:101C400001F0FCFD04220F4B21001A700E480C32EB
:101C500005F0DEFF102221000C4805F0D9FF072215
:101C60000B4B1C600B4B1C700B4B1C700B4B1A70FE
:101C70000B4B1C7010BDC046EE66FF1FED66FF1FCC
:101C80002045FF1FEC66FF1FDC66FF1FCC66FF1FB1
:101C9000C866FF1F9A66FF1F9966FF1F2245FF1F38
:101CA0009866FF1FF8B5174C0600257806A814247F
:101CB0000078052D23D1B41F134FA5B21824BD42BF
:101CC0001DD88D1FADB2BD4219D8FA256D00AA42AC
:101CD00015D21D000D4F0A3DADB2BD420FD80C4CC0
:101CE00026800C4C21800C4900240A800B4A13806A
:101CF000FFF714FF0A4B0421187806F0C1F8200002
:101D0000F8BDC046ED66FF1F790C0000750C0000A1
:101D10001E45FF1F1C45FF1F1A45FF1F1845FF1FCB
:101D2000EE66FF1FF0B50BB20D0089B0002B00DB93
:101D300076E1A64E307805F0C3FE041E55D0037838
:101D4000A22B00D127E1D02B1AD0912B4AD1437876
:101D50000E2B47D19E4B82889A4243D19D4A83687D
:101D60001278052A3ED1032018567F283AD09A4B84
:101D70001B68002B36D05B68002B33D0984731E0CE
:101D8000807807282ED806F063F9042D1D44447985
:101D9000ADDD6378002B11D10622E11C8F4805F0E0
:101DA00097FE01218B4B19708D4B1A78002A5BD05E
:101DB0008C4B307801F0A8FB002855D00722854BCA
:101DC0001A7051E061780029F8D1E378002B11D026
:101DD000854A864B1278307801F096FB6070637804
:101DE000002BEBD1200005F023FE8020000268408C
:101DF00009B0F0BD774B1B78022BF3D0012130786E
:101E000006F006F90028EAD10121307805F0F0FF4C
:101E1000E5E76378002BD1D16E4F032807D13B78DB
:101E2000052B02D101333B701EE00223FBE7704B10
:101E30001A88704B0293002A0BD01B78002B03D01A
:101E40000121307805F05CFF3B78062B04D1013B83
:101E5000E9E7029B1A70F7E7042B41D10121029BAD
:101E60003078197005F0C4FF5B4B1B68002BB9D0AC
:101E70001B68002BB6D0574A10787FE76378554F20
:101E8000002B27D10622211D5B4805F021FE628927
:101E90005A4B5B491A80A2895A4B1A80E3890B80FE
:101EA0000521397058490A80584A1380228A584BB4
:101EB0001A80584B1B78012B09D11F2000F036FDEA
:101EC000FA22920042430421307805F019FF0022E3
:101ED000484B75E7312B00D070E70022454B1A7054
:101EE0000323A0E706220021434805F091FE0023CA
:101EF000454A04211380454A30781380444A1380B0
:101F000005F0BEFF0821307805F0BAFFA379083B41
:101F10005A4253412F4A03331370314B1B78002B25
:101F200006D0344B30781A78002A06D001F02AFB0C
:101F30000122324B52421A8096E70121197005F0B6
:101F400057FFF5E70821307805F09AFF6378002BFA
:101F500000D047E72C4B2E4F0293E388029A0421CE
:101F600013802A4B307803932389039A1380638963
:101F70003B8006F04DF8002800D033E7264B1B6865
:101F8000002B00D12EE7039902983A88098800882F
:101F90001B68984726E74379132B00D022E7038973
:101FA000012B0AD11D4B1B78022B06D1082130785A
:101FB00005F066FFFFF726FE14E7052000F0B6FCEB
:101FC00008210200307805F09BFE0BE7EE66FF1F4C
:101FD00005140000ED66FF1F8066FF1FBF66FF1F30
:101FE0004845FF1F2945FF1FBA66FF1F9B66FF1F5D
:101FF000BC66FF1FBE66FF1F8D66FF1F2045FF1FCB
:102000009466FF1F9666FF1F8A66FF1F8866FF1F84
:102010008666FF1F8C66FF1F7C66FF1F8466FF1F9E
:102020008020C001014200D0E1E6CB0731D5324B20
:102030001B78002B1DD0314E05AC3378052B1AD1FF
:10204000023B23702E4B21001B7823722D4B1B78F3
:1020500063722D4B187801F0FBF9002809D0072096
:102060002A4B30701B68002B03D01B68002B00D05C
:1020700098470120BBE60E20254B06221B782549F8
:102080002370254B1B78637002ABC01805F020FD50
:10209000D8E7022308001840194209D0174B1B78D3
:1020A000052B03D11D4B188805F00AFF02209EE680
:1020B0000424214203D0FFF731FD200097E60823D6
:1020C00008001840194200D192E6154B1C78012CEB
:1020D00003D0022C0DD0082089E6124B124A134976
:1020E00013481B881288098800880094FFF7DAFDDE
:1020F000F1E7FFF787FDEEE7BE66FF1FED66FF1F06
:102100002245FF1F9866FF1FEE66FF1F8066FF1FB8
:102110009A66FF1F2345FF1F9966FF1F2045FF1F7B
:102120008466FF1F1845FF1F1A45FF1F1C45FF1F30
:102130001E45FF1F10B502A804880B20002C10D1EB
:10214000496808784978090201430C48814209D15D
:10215000022119800A4B59881170DB7800205BB28C
:10216000537010BD074C0A20A142FAD102211980F8
:10217000034B998811705B79F0E7C0466E2A000026
:102180009C64FF1F6F2A0000F7B5150008AA168887
:102190004A680F4F14785278120222430A24BA4236
:1021A00014D10122DBB2019200962A0005F0A0FBB7
:1021B000041E0BD1074B1B68002B07D068782A78C8
:1021C0000002104342425041013098472000FEBDBA
:1021D000022900000067FF1F30B5012503790400C4
:1021E000BFB02B4227D01549408804F0EDFE2842AD
:1021F0000DD06A46124B69465B8D138002235380D3
:10220000104B5B8893806088002201F09FFF0E498D
:10221000608804F0D9FEC0070DD56A460B4B6946AD
:102220001B88138002235380064B9B889380608811
:10223000002201F08BFF3FB030BDC046F866FF1FA3
:102240004C45FF1F9C64FF1FF066FF1FA645FF1F44
:1022500010B5074C0749200004F06CFE2000064929
:1022600004F068FE0721054A054804F025FE10BD6C
:10227000FFFF0000F866FF1FF066FF1FE4810211F8
:102280004C45FF1F10B5024802F0E6FD10BDC046E8
:10229000D921021110B5034C0B000122210000F0DE
:1022A0006BFA10BD552402110B8870B506000D00A5
:1022B0000224162B11D92B000322094900F05CFAE5
:1022C000041E0AD1074B2A881B88191C934200D987
:1022D000111C300089B200F0EFFA200070BDC0463A
:1022E000812402115E67FF1F10B54A780400013A8D
:1022F0000B000220012A07D80A78002A04D0052200
:102300002000024900F038FA10BDC046AF24021187
:102310000A7810B50B0004000220002A04D007221E
:102320002000024900F028FA10BDC0465B250211CA
:102330000A7810B50B0004000220002A04D00922FC
:102340002000024900F018FA10BDC046C125021154
:1023500010B5034C0B000B22210000F00DFA10BD4C
:10236000F125021110B5034C0B000D22210000F0E5
:1023700003FA10BD6326021110B5034C0B000F22A7
:10238000210000F0F9F910BDBD2602110A7810B540
:102390000B0004000220002A04D011222000024970
:1023A00000F0EAF910BDC046CD260211002310B599
:1023B0001322190000F0E0F910BD000010B5034C25
:1023C0000B001722210000F0D7F910BD1F270211C2
:1023D000002310B51922190000F0CEF910BD00003D
:1023E00010B5034C0B001B22210000F0C5F910BDF5
:1023F00059270211F7B584890D0006000121002C30
:1024000022D000238268D3561778002B1EDA0C2CBA
:102410001AD90C3CA4B2131940880093230002F08F
:1024200076FE431E984101307B06DB0F6B703F2325
:10243000013C1F40A4B22870AF70AC80002C07D0C4
:10244000B3680133AB6000210800FEBD0020EBE75C
:10245000AC60F8E70B7803704B8843704B881B0A1D
:1024600083700B79C370042070470420022B06D1BF
:102470000020537811781B02009A0B431380704799
:102480000B8803700B881B0A4370022070470420DE
:10249000009983420AD1537810781B0203430B80C2
:1024A000D37890781B02034300204B807047F8B527
:1024B0000D004B7801240021461C03702B788B42C1
:1024C00001D82000F8BD6B78B01C4F1C012B10D137
:1024D000890069184B88022233704B88B9001B0AA7
:1024E0007370691805F0F4FA04360434A4B2F9B232
:1024F000E4E7122359436B185A88043132705B8821
:1025000010221B0A7370691805F0E2FA12361234B1
:10251000ECE770B5049D14001E00052B01D80420C3
:1025200070BD637812781B0213432B80E378A27886
:102530001B02134302226B802A71211D681D063E77
:1025400005F0C6FAB2B22A81F02AE8D82800A11D07
:102550000A3005F0BDFA0020E2E7002310B50A7842
:102560009A4201D8900010BD9A008A18548801330D
:1025700004705488DBB2240A447094888470928872
:10258000120AC2700430EAE710B51100029C062B53
:1025900004D004201022142B01D010BD022222717D
:1025A0004B7808781B0203432380CB7888781B0282
:1025B000034363800431601D05F08AFA0020ECE7D4
:1025C00010B50C788B7804315C43E4B203702200C0
:1025D000013005F07DFA601C10BD0420022B06D1ED
:1025E0000020537811781B02009A0B431380704728
:1025F00010B50C000A88023105F06AFA208810BD77
:1026000070B504000D0004981100012B01D80420BE
:1026100070BD167852781202324302800200F832FE
:1026200055701470E825002C00D10C35023B9AB28D
:102630004280AA42EBD80231043005F049FA00206A
:10264000E6E70420009983420AD1537810781B02F0
:1026500003430B80D37890781B02034300204B8008
:10266000704710B50C000A88023105F031FA208855
:1026700010BD000070B501211E000420049C0E4016
:102680000B4218D1CB40DDB28D4214D90A49DBB2DE
:10269000098899420FD32300F6331D703300580088
:1026A00011184978165C0902314301332152D9B21D
:1026B0008D42F4D8002070BDC845FF1F10B50C0036
:1026C0000A88023105F004FA208810BD10B50C7894
:1026D0008B7804315C43E4B203702200013005F0D2
:1026E000F7F9601C10BD10B511000298032B01D83A
:1026F000042010BD14785278043B12022243028059
:10270000CA788C781202224342809AB28280F22ADE
:10271000EED80431063005F0DBF90020E9E710B50A
:102720000C000B8803700B881B0A43704B88837066
:102730004B881B0AC3708A880430063105F0C8F93B
:10274000A088043080B210BD0420012B03D10020EA
:102750001378009A1370704710B50C000B88037043
:102760000B881B0A43704A880230043105F0B0F927
:102770006088023080B210BDF0B589B003931E4B63
:10278000029242000700D05A019102F010F813257E
:10279000061E2DD0029B01240370019B002B04D048
:1027A000001903999847001984B26B461B7A5BB2F3
:1027B000002B0FDA1021380002F00CFB192500283D
:1027C00013D130003219E1B202F056FC051E0CD1D3
:1027D0000C34A4B2042304AA380005A993800696F9
:1027E000948101F09FFD051E02D0300005F0F0F944
:1027F000280009B0F0BDC0465C67FF1F70B505003A
:102800000C0000280CD00020814209D010222000AA
:10281000044905F05DF901202B7823736B7863730D
:1028200070BDC046FE810211F0B506000D00170014
:102830001C0085B002291BD00020102907D1022BD3
:1028400007D0102B03D115E00020102C08D005B0C4
:10285000F0BD69463800FFF7D1FF2A0069460BE05A
:1028600069463000FFF7CAFF22006946380004E0DD
:10287000022BE9D12A003900300005F059FAE6E7C9
:10288000031CF72800D9F723032008499AB2013A1C
:102890000B80D317034006499B189B100B80D30F66
:1028A00004499B185B100B807047C046CC45FF1F46
:1028B000CA45FF1FC845FF1F034B1B888B4202D32D
:1028C000024B4000C1527047CC45FF1F5C67FF1FA1
:1028D000014B4000185A70475C67FF1F1722014BDD
:1028E0001A8070475C67FF1F70B505000E2005F069
:1028F00037F9041E13D0D0230370002306228370FF
:1029000007494570033005F0E3F8064B2100DA8AE9
:1029100062811B7E2373044B187805F099FA70BD11
:102920007867FF1F6867FF1F1C46FF1F262803D814
:10293000024B4000C05A70470148FCE7CE45FF1FDC
:10294000FFFF000070B506000C00094D1C2200219D
:10295000280005F05DF9074B1E70074B1C7005F051
:1029600047FB0123002801D0002312202B7070BDEB
:102970006867FF1F1C46FF1F8967FF1F70B50500B2
:102980000D4C0800E260A16010220021656005F096
:10299000A7FA012803D11021A06802F048FD1022F7
:1029A0000021280005F09CFA012803D1102160685D
:1029B00002F03DFD70BDC0466867FF1F70B5041E84
:1029C00005D1002903D006220D4805F081F80D4BF2
:1029D0001D78012D11D1002C05D102221A7005F0AD
:1029E00017FA280070BD00221A70074B1B78FF2BC6
:1029F000F7D02000FFF778FFF3E70025F1E7C046A6
:102A00007867FF1F6867FF1F1C46FF1F030010B594
:102A1000002801D1002010BD00780B4A002803D106
:102A20005988D1821B7913761378022BF2D10023B7
:102A3000984200D103331370044B1B78FF2B01D055
:102A4000FFF752FF0120E6E76867FF1F1C46FF1FE4
:102A5000002911D000280CD04B79012803D1402245
:102A60005242134303E03F221340032802D00120C7
:102A70004B7170474022F4E70800FAE770B5094D42
:102A80000100287800280BD0074C0622200005F012
:102A90001FF821002878FFF7DBFF200005F078F908
:102AA00070BDC0468867FF1F6267FF1F00290AD0FC
:102AB000012808D13F224B799343C02B03D0403BE0
:102AC0005A425341981C704770B5174D06002B7839
:102AD000FF2B15D00A2005F043F8041E10D0D02398
:102AE0000370C83B8370114B11491B784670C3704B
:102AF0000622043004F0ECFF2100287805F0A8F944
:102B00000C4B1B78012B0DD10B4B1B68002B03D0FA
:102B10009B68002B00D09847084B04211878084A7E
:102B200004F0B6FF70BDC0461C46FF1F8867FF1F3C
:102B30006267FF1F8467FF1FB067FF1FB467FF1F37
:102B400060EA0000014B98687047C0466867FF1F45
:102B5000014BDB68186870476867FF1F074B10B5AB
:102B6000DA68136801331360054B1878FF2803D027
:102B70008021C90105F03CF910BDC0466867FF1F00
:102B80001C46FF1FF7B50E0002F0B8F8051E1CD05A
:102B90000E4B06621F78002F00D10778AB7910200A
:102BA000019304F0DDFF041E0FD0D0230380C73B48
:102BB0008370019BE91DC3700622043004F088FF76
:102BC00021003800E66005F043F9F7BD1A46FF1F03
:102BD000014B18787047C0468867FF1F054B0028D7
:102BE00005D1054B1A78054B002A00D1014B18007E
:102BF0007047C0467867FF1F8867FF1F6267FF1F27
:102C0000014B58687047C0466867FF1F024B186841
:102C1000431E9841C0B270478C67FF1F421E0300DD
:102C20000120152A03D9FF3B5A425341D8B27047BD
:102C3000F0B51C0000230E0085B0039002920B70CB
:102C4000029A934201D3002019E0E55C5A1CD2B2EB
:102C5000002DF8D0029851198142F4DC0233DFB222
:102C6000A35C18000193FFF7D9FF002807D0013DAE
:102C7000019A0399EBB233708A4202D1E01905B090
:102C8000F0BDDB19DBB2DBE710B50C0002F08EF80B
:102C900003001220002B03D02100588805F0A0F873
:102CA00010BD000070B50E4D84006359002B15D087
:102CB000186A002801D005F0C3F82B59586A00287B
:102CC00001D005F0BDF82B59986A002801D005F015
:102CD000B7F8285905F0B4F800232B5170BDC04651
:102CE0009867FF1F1C4B70B504000E001500994239
:102CF0000AD11A4B1B68002B01D1122070BD1B6832
:102D0000002BFAD09847F9E7154B994215D1134B90
:102D10001B68002B0AD01B68002B07D0984700289F
:102D200004D1104B1C70104B1D70E7E729002000E8
:102D3000FFF7AAFF0028E1D1F3E7080001F0DEFF6A
:102D40000028DAD003780320A342D7D1290030002D
:102D500005F046F8D2E7C046FEFF00009467FF1F6B
:102D6000FFFF00009167FF1F9067FF1FF7B504008A
:102D7000808801F0C3FF0025A84203D00578A08811
:102D800001F0F8FF1C4E3378002B1FD0AB421DD151
:102D90001A4B28001978FFF777FF002818D0002376
:102DA0003370A3790820A778A688019304F0D8FE91
:102DB000011E0DD0D0230370CA3B8370019B477066
:102DC00086808371280005F043F801E0002DE8D1EA
:102DD000A0880B4B8200D358002B01D0FFF762FF75
:102DE0001721A088FFF768FDA08801F017FDA088D3
:102DF00001F0EEFDF7BDC0469167FF1F9067FF1F12
:102E00009867FF1FF0B587B01D000CAB1B8807004B
:102E100001930DAB1B88142002930EAB1B88160088
:102E200003930FAB1B880091049310AB1B88059391
:102E300004F096FE041E1AD0D0230370CB3B4770DB
:102E40008370C670062229000430002D11D004F0D2
:102E50003FFE019B21006381029B0098A381039B9D
:102E6000E381049B2382059BA37404F0F1FF07B068
:102E7000F0BD04F0CDFEECE7F7B5009308AB1B887E
:102E800007000C200D001600019304F069FE041EDB
:102E900013D0280001F032FF00280FD00078D02393
:102EA0002370C93BA370009B21002381019B6770A5
:102EB000A580E680638104F0CBFFF7BD014B187855
:102EC000EDE7C0461C46FF1F13B504006489038963
:102ED000C2888188C0780094FFF7CEFF13BD000040
:102EE00010B5044C2068002803D004F0A9FF00238B
:102EF000236010BD9C67FF1FA122F0B5818892005E
:102F00004A43384B384F1B6804009B189D2292009F
:102F10009B18827989B01A603B68002B5FD01D78BE
:102F2000324B1B68002B04D05B68002B01D00020C3
:102F30009847260008363100E079FFF7B7FD237D7A
:102F4000E0710200E0780493638A29000393238AE6
:102F50000293E3890193A38800933300FFF752FFA4
:102F6000E378002B0BD1E289A379A1880292019624
:102F7000E27928000092012201F0CAFEE0703B686D
:102F8000002B20D0FFF7ACFF194D287800281AD06D
:102F9000184B1978FFF778FE002814D02B78E678C4
:102FA00008200793A78804F0DBFD011E09D0D02379
:102FB0000370CA3B4670837087808671079804F05F
:102FC00047FF00232B701721A088FFF775FCA0880E
:102FD00001F024FCA08801F0FBFC09B0F0BD064B19
:102FE0009DE7C0463409FF1F9C67FF1FB067FF1FA6
:102FF0009167FF1F9067FF1F1C46FF1FF8B5070072
:1030000008000E0001F07AFE041E18D02620FFF7FB
:103010008DFC051E00D12578062004F0A1FD041EBC
:103020000DD00021062204F0F3FDD0232370C23B13
:1030300021006770A370A680E8B204F009FFF8BD14
:10304000F0B585B001930AAB1B78070002930BAB78
:103050001B7808000D000092039301F04FFE061E3E
:1030600022D0102004F07CFD041E1DD0102200216F
:1030700004F0CEFD2620FFF759FC002800D130785F
:10308000D0232370C13BA370009B21002372019BBE
:1030900067706372029BA580A372039BC0B2E37248
:1030A0000C9BE36004F0D4FE05B0F0BDF7B50D0055
:1030B000019001F023FE071E20D00E2004F050FDE9
:1030C000041E1BD02620FFF731FC061E00D13E78DF
:1030D000D0232380C53B0622A370F91DE01C04F019
:1030E000F7FC019B2A0063810123DD401A401D404B
:1030F000210022736573F0B204F0AAFEF7BD000050
:10310000F0B585B0029010000D0017000A9E0393E1
:1031100001F0F4FD041E31D0029B002B2ED1039B45
:1031200002795B0724D5122313430422002E08D111
:103130000B99002905D10C99002902D10D9900297C
:103140001AD01A430D9B2271002B00D0C9E0002E2B
:1031500000D1CFE0002D00D0CCE0606A002801D083
:1031600004F06EFE1C21300004F04AFF606205E0AE
:1031700002239A430E33D7E793432371654BBA007A
:10318000D458002C00D1AAE0002E10D0236A002BC6
:1031900003D11C2004F0ACFD20625E4BBA00D35872
:1031A000186A002803D01C22310004F091FC0C9B0B
:1031B000002B12D0574CBB001D596B6A002B03D15A
:1031C000162004F095FD6862BB00E358586A002899
:1031D00003D016220C9904F07BFC0D9B002B11D020
:1031E0004C4DBC006659B36A002B03D1142004F087
:1031F0007FFDB0622B59986A002803D014220D99E4
:1032000004F066FC380001F079FD051E67D0414BE3
:10321000BA00D358002B62D01A6A3420002A00D199
:103220001C389A6A002A01D0143080B20B9A002A06
:1032300001D01C3080B25B6A002B01D0163080B206
:1032400004F08EFC041E4AD01822002104F0E0FC99
:103250002620FFF76BFB0190002801D12B7801930A
:10326000D0232370029B200063700A23294EA37091
:10327000039BBD00A371AB59A780196A18300029C0
:1032800005D01C22A06004F023FC200034307359C8
:10329000996A002907D0030014221433E0600293D6
:1032A00004F016FC02980B9B002B08D003001C2294
:1032B0001C330B992061029304F00AFC02987359A5
:1032C000596A002903D01622606104F001FC6B46A4
:1032D0002100187904F0BCFD3800FFF7E3FC05B0CD
:1032E000F0BD10220D9B0D991B69A018236204F0FC
:1032F000EFFB2CE70B9B002B00D13FE7012D00D00B
:103300003CE7606A002801D004F09AFD1C210B986C
:103310002AE7C0469867FF1F10B5044C20680028B4
:1033200003D004F08DFD0023236010BD8C67FF1FC8
:103330000B4B07B51A68002A01D100200EBD694663
:10334000531C012012780731FFF772FC0028F4D0DB
:1033500002780123100018401A42EED0EEE7C04672
:10336000A867FF1FF0B51F4F01203B6887B0002BF7
:1033700025D09B78059300F0B3FB002821D00A20CC
:10338000FFF7D4FA04000B20FFF7D0FA164B050024
:103390001E78731E9E413B68F6B2191DD878FFF760
:1033A00057FB3B682900DA7A043303929A79019338
:1033B0000292009033002000059A04F079FD07B0D6
:1033C000F0BDFFF7B5FF002805D00620FFF7AEFAE5
:1033D00004000720D8E70820FFF7A8FA0400092016
:1033E000D2E7C0468C67FF1F8867FF1F70B50A4E83
:1033F000040033780D00FF2B0DD0042004F0B0FB47
:10340000011E08D0D0230370CE3B45708370C4707A
:10341000307804F01DFD70BD2C46FF1F70B5040010
:1034200006200D0004F09CFB011E0AD0D02303707F
:10343000CD3B8370054B44701B688580187804F081
:1034400007FD002C01D0FFF767FF70BD8C67FF1FE1
:10345000F8B5264F06003B680D001124002B05D15E
:103460000522234B1B78134202D112242000F8BD01
:10347000204A10241268002AF8D01278002AF5D0C9
:10348000DB0719D52B789A1E012A1AD80C2004F0D4
:103490002FFC132438600028E8D000230A22437050
:1034A00029000670023004F013FBFFF75BFF041ED7
:1034B0000AD0FFF731FFD9E700F012FB0028E1D175
:1034C000E4E7002BE2D0D0E70B4B1B78032BCDD1E8
:1034D0001D20FFF72BFA094B18800028C6D0084B97
:1034E00004211878074A04F0D3FABFE78C67FF1F5E
:1034F0008967FF1FA867FF1F8867FF1F8667FF1F79
:10350000B467FF1F60EA0000F7B50193194B140080
:103510001A78052306000F0012201A4221D0012933
:1035200020D1154B1D68002D1BD002201F2C18D850
:10353000002C02D0019B002B13D0104B1F221E70B9
:103540006E1C0021300004F063FB01992200300062
:1035500004F0BEFA310020002C70002F06D004F0D9
:10356000C7FCFEBD064B12201D68DCE704F070FAB4
:10357000F7E7C0468967FF1FA867FF1F2C46FF1F9C
:10358000A467FF1FF8B50F4E12243368002B17D025
:103590001B780F3C834213D100250B4F0221387852
:1035A00004F06EFC094B042138781D8004F068FC9F
:1035B000074B28001D8033685C7004F001FD040097
:1035C0002000F8BD8C67FF1FB467FF1FA067FF1FB7
:1035D0008667FF1F70B5012823D11B4C2388002B61
:1035E00003D01A4A1578002D07D0194B1B68002B01
:1035F00002D01878FFF7C6FF70BD3B2B02D93C3BC9
:103600002380F9E7134E0221307804F039FCFA22C6
:103610002388920002215A43307804F071FB258000
:10362000EAE70B4B1B68002BE6D00B4B1B785B07C4
:10363000E2D5084B0221187804F022FC0022024B4C
:103640001A80FFF769FED7E7A067FF1F8467FF1F97
:103650008C67FF1FB467FF1F8967FF1FF8B51E4DFA
:103660002868002803D004F0EBFB00232B601B4EDE
:103670003068002803D004F0E3FB00233360184FC8
:1036800005243B7818002040234221D0154800F043
:103690002BFA3B78234213D0202004F029FB28602A
:1036A000002813D02022002104F0B2FA202004F0D8
:1036B0001FFB041E306005D02022002104F0A8FA70
:1036C000002004E0286804F0BBFB2C601320F8BD48
:1036D00000F00AFAF4E7C046A867FF1FA467FF1FBF
:1036E0008967FF1F2046FF1F10B50A4C23681A1E6A
:1036F0000ED0002808D10130587004F061FC002879
:1037000005D02368002B02D00021FFF787FE01229D
:10371000100010BD8C67FF1FF7B5274E05003368FA
:103720000191181E21D05C78244F012C30D1FFF775
:10373000FFFD002825D02000FFF7F8F804004128FD
:1037400014D91F4B022118781E4A04F0A1F91E4B10
:103750003C3C1C80022233685A703B78002B14D109
:1037600028000199FFF75AFE0120FEBDFA229200BF
:103770004243002AEED0124B0221187804F0C0FA1E
:10378000E8E7FFF7D3F80200F3E700233B70EBE72D
:103790003B78002BE8D1032004F0E2F9011E08D0A9
:1037A000D0230370CC3B457083703368187804F0E5
:1037B0004FFBFFF7B1FDD7E78C67FF1F8467FF1F43
:1037C000B467FF1F60EA0000A067FF1F10B517492C
:1037D000838802008B4220D011D815498B4217D024
:1037E000144900205B1899B2012907D89268117812
:1037F0005A425341D8B2FFF7F9FD012010BD0E4ADD
:1038000000209B1807229BB29A424041C0B2F5E7C4
:1038100083681878FFF768FFF0E7836899785A782B
:10382000090218781143FFF777FFE7E70A20000045
:1038300006200000F8DFFFFFAFDFFFFF014B18702D
:103840007047C0462D46FF1F10B5064C207001F092
:1038500031FA207804F064FA0521207800F052FD56
:1038600010BDC046B467FF1F0BB273B50D00002B2F
:1038700000DBC4E0884B187804F022F9041E0ED057
:103880000378912B0FD0A22B00D1A1E0834B1878A5
:10389000FF2852D0210004F0DBFA00284DD180200F
:1038A0000002684076BD43780F2B76D013D8052BE5
:1038B00070D00E2BEAD18088794B98422BD8794B67
:1038C00098421BD8784B9842E0D1A3681878591CCD
:1038D000FFF774F838E03E2BD8D18378032B74D0EF
:1038E0006CD8012B6ED0022BD0D1704B1B68002BF3
:1038F00023D05B68002B20D098471EE06C4BC0188B
:103900000C28C3D804F04CFA1DC2C2150BC20B0B15
:103910000B3223C23C00674BC0180728B6D8664B51
:103920001B68002B09D01B68002B06D0200098478D
:103930000AE0A3681878FFF7C7F8200004F078F8C9
:10394000ADE7A068FFF762F800289FD0F5E7A3680D
:103950001B78002BF1D0554B1B68002BEDD01B685A
:10396000002BEAD0210055489847EDE74F4B1B68E4
:10397000002BE2D01B68002BDFD021005048F3E77A
:10398000504B1B68002BD8D05B68002BD5D0210092
:103990004348E9E7FFF7EAF9CFE780884A4B9842C6
:1039A00003D04A4B984200D070E7464B1B68002B6F
:1039B000C3D05B68002BC0D02100D5E7153B012B9D
:1039C000BBD963E7FFF798FAB7E7FFF77DFAB4E7EB
:1039D0003F4B1B78042B07D100236A4613800179E3
:1039E000408800F0B5FCA8E7364B1B68002BA4D03C
:1039F0005B68002BA1D00100364898479DE7012461
:103A000021420AD0294B1B68002B04D05B68002B95
:103A100001D000209847012043E78B070AD5264BA9
:103A20001B68002B04D05B68002B01D02000984756
:103A3000022036E70421280008400D4200D131E77A
:103A4000254E3388002B21D0013B9BB23380002BC5
:103A50001AD1FFF7DBF800280AD0204B1C70164B58
:103A60001B68002B04D05B68002B01D02000984716
:103A7000FFF7C6F8694601F0F1FC6846FEF7FEFF65
:103A80001D20FEF753FF308004200AE7024B187810
:103A900004F0F6F9F8E7C046B467FF1F2D46FF1F94
:103AA0000E2000000120000009100000AC67FF1F7D
:103AB000FEDFFFFFAFDFFFFFB067FF1F0C2000003E
:103AC0000B2000009467FF1F0D2000001320000052
:103AD0008967FF1FFFFF00008667FF1F8467FF1FC6
:103AE00010B501F08BF910BD014B18607047C0464E
:103AF000B067FF1F0B880020162B01D81723042066
:103B0000014A13807047C0465E67FF1F0020704760
:103B1000074A03001188814207D09188002099420A
:103B200002D101308000101870470020FAE7C0462B
:103B3000BC67FF1FF0B58F7806000D00C7B01E2FC1
:103B400015D1FFF7E5FF051E03D10024200047B083
:103B5000F0BD00223B003100C078009200F0A2FBD3
:103B60000400A81C00F0C3FBFF23EB70EEE7264B1C
:103B7000062403931B78FF2BE8D0182FE6D87B0888
:103B8000224A013BDB0002929A589446002ADDD07B
:103B9000029AD3185B68002BD8D00878002802D18D
:103BA0004B78012B02D10624122FCFD107AFAB885F
:103BB000697800976446AA68A047041EC6D1AB780E
:103BC000029A5B08013BDB00D318390030005B68C8
:103BD0009847041E0BD1AB78042BB6D0039A310062
:103BE00010782200009700F05DFB0400AEE76A78D1
:103BF000002AABD1AA7805A93B88087130000A7069
:103C00004B80FEF747FBA0E73046FF1F10820211F2
:103C10001D4B37B5050098420BD000290AD1FFF79C
:103C200077FF002805D11948FFF772FF002800D060
:103C3000058037BD01291AD1FFF76AFF041EF8D0AD
:103C400001235B420380A378FF2BF2D0FE2B07D029
:103C50000023E0781422009329001E3300F022FB99
:103C6000A01C00F044FB01235B426380E1E70229D2
:103C7000DFD1013901F0AEF80028DAD12800FFF7D2
:103C800047FF041EDFD1D4E7FEFF0000FFFF000066
:103C9000022210B5074B52421A80074801325A805F
:103CA0009A80DA8000F06EFA044801F015F80020DE
:103CB00010BDC046BC67FF1F353B0211113C02110D
:103CC0000388F7B50400002B02D102252800FEBDB1
:103CD00042680221137825485268FEF7A5FD0028A6
:103CE0002ED0234F01253A88002AEFD08023218847
:103CF0005B0201259B1A9942E8DC0C2003F0F8FFD7
:103D0000061E31D03B8822889C460023180001956E
:103D100061469DB2491989B2AA421BD8002801D038
:103D200062443A8000233000082208C0210003F0DA
:103D3000CFFE104A1368002B13D100251660C5E78B
:103D40006268022113780C485268FEF76DFD002866
:103D5000C7D1BAE760681D0140194181013301985C
:103D6000D6E71A001B68E6E71325AFE77E8202114B
:103D70002E46FF1FB867FF1F7C820211014B18708F
:103D80007047C0463046FF1F14230A0010B51A4082
:103D9000194204D00122102101F038F810BD4B0661
:103DA000F9D4012088434000F8E710B514008B06D1
:103DB00004D50122102101F029F810BD08230A00C2
:103DC0001A40194202D14BB2002B0FDA102101F038
:103DD0001DF8002808D02300F9331B78002BECD005
:103DE000F8342378012BE8D10020E6E70320890787
:103DF000FAD4E2E7F0B51F00184B85B01C680190BB
:103E000002910392002C27D1200005B0F0BDA568D7
:103E10003301ED186B89019A934211D3029A9342B0
:103E20000ED8002F04D10A9B002B10D12C00EBE7F9
:103E30003B002978039A6868FEF7F6FC0028F2D167
:103E40000136B6B2A388B342E1D82468DAE7A368A2
:103E50000A9A5B891380E9E70026F3E7B867FF1F3A
:103E600037B50C000A8849880123914217D3002AEC
:103E700015D0651D23792A0002210A48FEF7D4FCDB
:103E8000102300280BD023796188208800242A0081
:103E90000094FFF7AFFF0A23A04200D023001800D0
:103EA0003EBDC0467E82021113B50A0008884988CB
:103EB000012388420BD8002809D000241379053249
:103EC0000094FFF797FF0A23A04200D023001800B8
:103ED00016BD13B50A0008884988012388420BD80B
:103EE000002809D00024137905320094FFF782FFDF
:103EF0000A23A04200D02300180016BDF0B58BB0F5
:103F000003904A8808880E000123824255D3002876
:103F100053D00023012704AC2370002271881300C2
:103F20000092FFF767FF051E3ED02078002835D1AC
:103F30002B78022B18D167706A8983000130E3184F
:103F400080005A8069680222201803F0C1FD23789E
:103F50000133DBB22370042B19D93B00688901308F
:103F600080B2002BD9D01FE0022363701223584384
:103F70006A89231804305A8069681022201803F0D7
:103F8000A7FD23780133DBB22370002BE5D10C4A67
:103F90006B899B185A425341DBB2DFE76378012BF0
:103FA000E4D12B78022BC7D022780A23002A04D030
:103FB00021000398FEF798F9002318000BB0F0BD1C
:103FC0000100FFFF0F4BF0B504001868002816D061
:103FD00083685D89A54207D88288AE18B44203DAA7
:103FE00012019A18934201D10068EFE71E005F8921
:103FF0001036A74204D1002900D00D801800F0BD72
:104000003300EFE7B867FF1F70B505000C000888A4
:104010000021FFF7D7FF03000120002B04D022006E
:104020002800197AFFF7C1FE70BDF7B50C00002516
:1040300001902300F6331B78AB4201D800200AE040
:104040006B00E65A00213000E718FFF7BBFF00289D
:1040500002D126800130FEBD017A0198FFF794FE5F
:10406000002802D03B882380F5E70135EDB2E0E778
:1040700010B5040008880021FFF7A4FF0300012009
:10408000002B03D02000197AFFF77EFE10BD000040
:10409000054B1B68002B01D1180004E09A68528977
:1040A0008242F6D198887047B867FF1FF0B50E2797
:1040B000002687B0039302ABFF183E8005001F4B1C
:1040C00040891400984207D02B78013000976A6825
:1040D00080B2FFF78FFE060002212B7818486A682D
:1040E000FEF7A2FB00280FD06C892000FFF7D0FF5D
:1040F000002802D0013C0419A4B2039B002B00D07D
:104100001C80300007B0F0BD02212B780D486A6892
:10411000FEF78AFB0028E7D102212B780A486A685B
:10412000FEF782FB002807D0002EDED03B88A3429A
:10413000DBD17489013CDFE76C89DEE7FFFF00001B
:104140007E8202117C8202117A82021170B5040013
:104150000D001600FFF7DCFC002803D08378172041
:10416000FE2B05D0002E04D129002000FEF738F9DF
:1041700070BD01221021200000F048FE0028F3D07D
:10418000F6E70000014B18607047C046C867FF1F84
:1041900037B56B469D1D010004000222280003F084
:1041A0006FFD2B88B02B0ED12379122B09D1230060
:1041B000FF339B78012B06D10121608800F0E0F8E5
:1041C00001E01B2BF8D037BD10B5054B042118704A
:1041D00000F098F8FFF75CFDFEF780FB10BDC046CD
:1041E000CC67FF1F0020F0B50BB20F0087B08342F1
:1041F00034DA274B187803F063FC051E2BD00378C4
:10420000A02B25D103AE3100FEF7F4F8041E0BD12C
:10421000B378DB0724D51F4B06341B68002B03D073
:104220003100688898470400A868002801D003F08E
:10423000CFFC002C08D1184A039B1340174A934225
:1042400006D0B3781B2B03D00121688800F098F8C2
:10425000280003F0EDFB80200002784007B0F0BD9D
:104260000F4B1B68002B10D0310068889847041E44
:10427000DAD07378002BD7D1B27801A90A704B80BD
:104280000C716888FEF706F8CEE70624F1E7C04611
:10429000CC67FF1FC467FF1F00FFFF000001120073
:1042A000C867FF1FF7B50190822040000D0017007E
:1042B0001E0003F055FC04001320002C12D0B02384
:1042C00020002370089BFC226770658026710830EF
:1042D000002B08D0190003F0FBFB2100019803F02C
:1042E000B7FD0020FEBD089903F092FCF5E710B57C
:1042F000041E06D00078FD2803D803F039FCFF2304
:10430000237010BD0A1F93B210B504000220032BC6
:1043100005D882400020024BD1529B189C7010BDE2
:10432000EC67FF1F0B8870B5043B04000D000220F2
:10433000032B0BD80121200000F04CFD03001420BA
:10434000002B03D02900200000F0DEFB70BD000030
:1043500007B51300034A00920A00012100F02CFC6B
:104360000EBDC0468D45021107B501920322009291
:10437000024B0A00122100F049FC0EBD0B4602114F
:1043800007B56B4601AA11800449D8800878063326
:10439000012802D1190003F0A3FC07BDCD67FF1F60
:1043A0000C4B10B518700023FF210B4A13801381AA
:1043B00093819380094A5380137051729381937251
:1043C000D174D3821375517703F0BAFD00F0FCF974
:1043D00010BDC046FC67FF1FEC67FF1FCE67FF1FC5
:1043E000F0B58DB06B46002003910C229B5E83429A
:1043F00000DBB0E05D4B187803F062FB051E00D1D6
:10440000A4E00378902B00D09DE006AF0100468821
:10441000380000F013FA79680400002900D19CE00C
:104420003B88052B6ED13B89032B1CD905AC2000A2
:1044300000F0A2F86288172A61D83989131D9942C1
:1044400031D17968237804310291D90738D5607861
:1044500000F08EF9071E06D0002303712378012B8C
:1044600008D0132B23D0A868002800D178E003F0EF
:10447000AFFB75E06288029909A800F0A6F80290E7
:10448000380000F08BF909AA2378387A01920022CB
:1044900031000092029A00F012F9380000F064F93D
:1044A000029B002BDFD0300000F080F9DBE70378BF
:1044B000032BD8D16288029909A800F0D6F8DEE76C
:1044C000122B13D1029909A800F0B5F8021EEAD107
:1044D00027498B88002BC6D0887909A923780191B8
:1044E00061780091310000F0EAF8BCE7002302AAED
:1044F00093833000617809AAFFF72AFFB3E71D4BC9
:104500000993F6E7042B02D09A1F012AABD8184A68
:10451000043B9B00995A0029A5D0D218907831000D
:104520003A0000F0AEF800289DD13B88042B03D060
:1045300001213000FFF724FF012C04D1A8680028D6
:1045400001D003F045FB280003F072FA8020039BA2
:104550000002434018000DB0F0BD012800D182E7F1
:1045600001213000FFF70CFFEDE7C046FC67FF1F9D
:10457000EC67FF1F010017000B7803704B78437046
:10458000CB788A781B021343438070470A88030064
:1045900002700A88120A42700A88012A06D14A88E3
:1045A00082704A88120AC270042070470220824238
:1045B000FBD14A8804309A704A88120ADA708A88D5
:1045C0001A718A88120A5A71EFE710B504000120A7
:1045D00082420CD94B780A781B0213432380834212
:1045E00006D1CB788A781B0213436380002010BD6C
:1045F000022BFBD1CB788A781B02134363804B7963
:104600000A791B021343A380F0E70B8803700B8821
:104610001B0A43704B8883704B881B0AC3708B88BE
:1046200003718B881B0A4371CB888371CB881B0A6B
:10463000C3710820704703000120082A14D14A786A
:104640000878120202431A80CA788878120202435C
:104650005A804A790879120202439A80CA79887985
:10466000120202430020DA80704710B504000120D6
:10467000022A05D100204B780A781B0213432380BD
:1046800010BDF8B5060010200F00150003F068FA01
:1046900004000120002C0ED0A0230C22290023802E
:1046A0006780201D002D07D003F012FA2100300092
:1046B00003F0CEFB0020F8BD03F0AAFAF6E7F7B549
:1046C0001E00009008AB142017001D78019103F024
:1046D00047FA041E12D0A2230370019B4770438047
:1046E000099B057146710C220830002B07D0190078
:1046F00003F0EEF92100009803F0AAFBF7BD099939
:1047000003F086FAF6E737B5041E0FD04388002B76
:104710000CD00025C1881323007A1722019500953B
:10472000FFF7CDFFFF2365806372257037BD000062
:1047300010B50C4904004A88002A09D08B89002B47
:1047400005D00020CB8A0222834201D010BD012275
:1047500013000A20434300204032C854C818428046
:104760000472F3E7CE67FF1F002343800370704796
:10477000094B00211A0010B55C88002C06D01C796A
:10478000844203D10A234B43D01810BD01310A33B0
:104790000329F1D10020F8E7CE67FF1F10B5040010
:1047A000407A03F0E5F9FF23637210BD70470430CF
:1047B00010B580B203F0BCFB002803D004214942AD
:1047C00003F03EFC10BD000070B50025104CA06841
:1047D0002580A581A580A84202D003F0F9F9A56043
:1047E00000250C4C0C4B606D1D80230058331D7050
:1047F000A84202D003F0ECF9656500256068002846
:1048000001D003F0E5F9013508340A2DF6D170BD69
:104810009468FF1F3868FF1F8868FF1F70B5041E6B
:1048200009D1054D2880A881A880A868002802D059
:1048300003F0CEF9AC6070BD9468FF1FF0B54B88F3
:1048400085B00193002343600A7905000F00022A16
:1048500000D07BE0CA88032A17D98B685E78197864
:104860003602DC78D8790E4399781B7A24021B0231
:104870000C43034353495BBA0B80331D93421ED153
:10488000042C04D0631F022B0ED9012015E0019ADD
:104890004D4B1201D35A002B06D00198FFF7BEFFF3
:1048A0004A4A1369013313610421B8682E812C80B0
:1048B000494203F0C5FB6860002005B0F0BD434DE0
:1048C000042C06D0631F022B0FD9EB680133EB6079
:1048D000DBE7019A3C4B1201D35A002B05D001981B
:1048E000FFF79CFF2B6901332B61374B300002939C
:1048F000019B029A1B010193002301998C468B5264
:10490000130063449C8003939E81FFF750FF039B39
:10491000041E986016D00421B868494203F090FB49
:10492000FA880100043A200003F0D2F80199029AB3
:10493000FB888A5A043B9B18029A8B522B680133DE
:104940002B60A2E7AB690133AB619EE71E4B02937C
:10495000019B1E01029BF35A002B2DD002998C194A
:10496000A068002828D0012A26D1FA889B189BB27B
:104970007352A189994217D39B1AC018B96803F0E2
:10498000A7F8029BA289F35A934200D07DE7002248
:104990002B81A3882B80A3686B60029BF2520B4A89
:1049A00053680133536070E7084A9368013393609A
:1049B0000198FFF733FF68E7044A536901335361F5
:1049C000F6E7C046FE67FF1F9468FF1F0468FF1FDD
:1049D00070B5051E15D10B4C0B4B188023005833B6
:1049E0001870606D002802D003F0F2F865652500AC
:1049F00050356068002801D003F0EAF80834AC4272
:104A0000F7D170BD3868FF1F8868FF1FF0B5170029
:104A1000A12285B0920001934243394B06001B68E6
:104A20000C009B18D933FF331D78FDF751FF04307C
:104A3000854204DD3000FDF74BFF0430C5B2BD42B6
:104A400007D33A0000213000019B02F0D9FF05B0E6
:104A5000F0BD2900380003F0ABF92300C6B2503393
:104A60001E700393019B29006365380003F000FA70
:104A7000CBB20293002B02D0039B01361E7000269E
:104A80002300503303931B78B34204D8606D002891
:104A900031D10020DBE7029A2800002A04D0013B34
:104AA0001000B34200D02800F700E719387003F077
:104AB0004FF9786000280ED03A78019903F008F891
:104AC000019A3B780136D3180E4A0193D369F6B2A6
:104AD0000133D361D4E7039B18706065A74205D109
:104AE000084A1320D36A0133D362B0E7606803F049
:104AF0006FF80834F2E703F06BF800236365C8E74A
:104B00003409FF1F0468FF1FF7B50D0007000421DB
:104B1000686803F095FA2B89040003702B891B0A3F
:104B200043702B8883702B881B0AC3702E89022543
:104B30000436F6B2FB2E15D81B4B9F4214D10C2025
:104B400003F00EF81135011E0CD0902303708E3B3C
:104B50000371043B4380154B8460C680187803F0D2
:104B600077F900252800FEBD5C237B43104AD3184B
:104B70000093583301931B78002B0FD103003200B0
:104B800038000099FFF742FF019B05001B78002BBE
:104B9000E8D13800009903F02BF8E3E7054A072530
:104BA000536A01335362DDE7FEFF0000FC67FF1F1D
:104BB0003868FF1F0468FF1FF0B587B0009017200A
:104BC0000F0016000193FFF7F2FD1325041E19D004
:104BD0000C98031E02D00199201D9847030AE37028
:104BE000052302AAA0700430908127700098667097
:104BF00003A993800494FFF787FF051E02D02000CD
:104C000002F0E6FF280007B0F0BD0000F0B587B065
:104C10001F000CAB1B780391059301210DAB06001F
:104C20001C78049200F0D6F81425002821D020002A
:104C3000FFF77EFD0135041E1BD01149059B0A7844
:104C400003700132D2B2131EC68001D101231A00B3
:104C50000B7022713000049B03990097FFF7ACFFA3
:104C6000051E09D1230021000648074A093302F036
:104C70003FFF280007B0F0BD002363802370F8E7F2
:104C80000068FF1F0747021130750000F8B50500E6
:104C90000E00064C064F2368002B02D0310028007E
:104CA00098470434BC42F6D1F8BDC046A468FF1F43
:104CB000B868FF1F0123064A5B425380002313712B
:104CC0005362044A136053609360D360136170476A
:104CD000B868FF1FA468FF1F0200002310B5064933
:104CE0009C000859002801D1625010BD0133052BEA
:104CF000F6D11320F9E7C046A468FF1F034A538882
:104D0000181A43425841404210407047B868FF1F8C
:104D1000F0B585B002930AAB1F780CAB1B880090EE
:104D200008000E0001920393FFF7E8FF0500112031
:104D3000002D1BD10E48FFF7E1FF04001520002CC9
:104D400014D006220B99A771E01D02F0C1FE019B51
:104D500030002371029B29006371009B66802370E1
:104D6000039B6562E381FFF791FF280005B0F0BD6A
:104D7000FFFF000010B5FFF7C1FF04000220002C68
:104D800012D060880121FFF781FF606A002801D0FE
:104D900003F056F828220021200002F039FF0123F9
:104DA00000205B426380207110BD000030B5074ACF
:104DB000074C5588010013780020A54204D05B1AE7
:104DC00059424B415842104030BDC046B868FF1FA1
:104DD000FFFF0000084A10B501230C00904208D0E4
:104DE000FFF78CFF031E04D0037923405A1E934122
:104DF000DBB2180010BDC046FEFF0000024B187960
:104E0000431E9841C0B27047B868FF1F70B50400D8
:104E10000D001600FFF772FF002804D10D4B9C42D5
:104E200000D0143070BD416A03790520002907D0F5
:104E300012221A40102A02D10520002EF2D10F2092
:104E4000DB06EFD5897E0C20A942894149424942BF
:104E50000840E7E7FEFF0000030010B5002800D17E
:104E600010BD0348034A41889142F9D09847F7E7BB
:104E7000B868FF1FFFFF0000002330B5C45CCD5CA5
:104E80006C40D4540133102BF8D130BD0F230022D5
:104E900010B5C45C64002243CA54C25CD209013B11
:104EA000F7D210BD0200010010B52032103102F01F
:104EB00027FE10BDF0B58BB00390102005931700AE
:104EC000049102F015FF0090102002F011FF009BEA
:104ED00013240190002B05D000280CD11324009836
:104EE00002F0AEFF019B002B02D0180002F0A8FFD9
:104EF00020000BB0F0BD102002F0FAFE06001020DA
:104F000002F0F6FE13240500002E00D1AEE00028CA
:104F100019D01022002102F07BFE320029000398F4
:104F200002F0EEFD041E0ED133787F2B51D83000F5
:104F30000099FFF7ABFF009B1B787F2B53D801999B
:104F40000098FFF7A3FF300002F07AFF002D02D097
:104F5000280002F075FF002CC1D1102002F0C8FE1D
:104F60000600102002F0C4FE0290002E7CD0002823
:104F700078D03A000F3223000125121105D00F33EB
:104F80003B4015B25A4253411BB26A1E1201002B1C
:104F900033D0049BD2B298180099029AFFF76CFFA5
:104FA000013D10220021300002F032FEADB2049F1C
:104FB0002D017D19AF4242D0002C33D0300002F0D9
:104FC0003FFF029B002B00D189E7180002F038FF59
:104FD00085E729003000FFF759FF28002549009A8E
:104FE000FFF74AFFA7E729000098FFF74FFF2800C7
:104FF0002049019AFFF740FFA5E70F210F400499D0
:105000008A18D9B28F4208D9D15C06A81954013345
:10501000102BF6D1029A0199C0E7791A4842414112
:10502000C901F2E73900300006AAFFF725FF320078
:10503000039806A902F064FD10370400BAE7002CBB
:10504000BCD13000029906AAFFF716FF320006A96C
:10505000039802F055FD082204003100059802F083
:1050600037FDABE71324A9E71324AAE7002800D0F3
:105070006EE733E784820211F0B58BB00F001600A3
:105080000225009000283FD0002A3DD00B1DDBB246
:105090001800029302F02CFE1135041E34D0FDF7E7
:1050A00057FD05003A000099201D02F049FEEBB2C1
:1050B0000393E3702B0CDBB22F0A00936370FFB2F3
:1050C0002B0E2370A7700193FDF73CFD1022010009
:1050D00006A802F035FE2100029A04AB06A8FFF7ED
:1050E000E9FE051E0DD1039B08223370009B04A925
:1050F000B370019B7770F370301D02F021FEFDF755
:105100002DFD200002F09CFE28000BB0F0BDF0B594
:105110008FB00D00149E039004920593002A03D1D2
:10512000022420000FB0F0BD002EF9D00398FFF745
:10513000E5FD1424071EF4D07278337812021A4366
:10514000B3781B041343F27812061A43036A0192E0
:10515000934201D30133E3D1002D03D03B790124E5
:105160009B07DED50822002106A802F051FD059B11
:1051700013240433DBB21800029302F0B9FD051EBC
:10518000CFD0059A0499043002F0DAFD04223100F0
:10519000280002F0D5FD3900102210310AA802F0D3
:1051A000CFFD2900029A06AB0AA8FFF783FE041E72
:1051B0000FD1082206A908A802F0C2FD0822311D5D
:1051C00008A802F0B5FD012807D101990398FDF761
:1051D000D9FC280002F034FEA3E70124F9E700001F
:1051E00070B51C4C05002368181E10D0002D14D17A
:1051F0001A78002A0CD1981C083202F069FC02F0DF
:1052000087FD0135002808D123681D70012070BD7D
:105210000A331800082202F05BFC2368002BF5D04B
:10522000122002F09DFC061E0DD0C12321680370E0
:10523000457002311022023002F04AFC236831002E
:10524000587802F005FE206802F0FAFD0023236082
:10525000DCE7C046E068FF1FF8B504002020FDF73A
:1052600065FB0D4EA700BB590500002B0DD0002893
:105270000BD0D878FF2809D108492A000C55F359DA
:1052800007480333611802F033FCF8BD290002F02F
:105290003FFE0028F0D1F8E7FC68FF1FE468FF1F1D
:1052A000B164021170B5064D84006359002B05D01E
:1052B000D87802F05DFCFF226359DA7070BDC046F9
:1052C000FC68FF1F70B506008CB00C0015000021B3
:1052D0003022684602F09CFC31001022684602F041
:1052E0002FFD1D2021000322684402F029FD68469D
:1052F000FFF7D8FD2D21040003222800694402F0A5
:105300001FFD20000CB070BDF0B50700160097B06F
:1053100001931CAB1D7830221EAB00910AA800211E
:105320001C7802F075FC102239000AA802F008FD72
:105330001022002102A802F06BFC0722310002A813
:1053400002F0FEFC072202AB9818631E9C410199F3
:1053500002F0F6FC02AB9C732B005A1E934102AA8A
:10536000D3730021102206A802F052FC06221D99D8
:1053700007A802F0E5FC1A2002ABC01806221F990C
:1053800002F0DEFC102200990EA802F0D9FC1022D7
:1053900002AB0EA908781C78013A6040D2B20870BE
:1053A00001330131002AF5D10AA8FFF77BFD102255
:1053B00012A904000EA802F08BFB102206AB0EA966
:1053C00008781D78013A6840D2B208700133013183
:1053D000002AF5D10AA8FFF765FD044310222098A2
:1053E000E4B212A902F0ACFC200017B0F0BD70B519
:1053F0000E0014008CB00100102268461D0002F05F
:105400009FFC3100082204A802F09AFC2100082227
:1054100006A802F095FC6846FFF744FD0400102240
:10542000280008A902F08CFC20000CB070BDF8B573
:1054300006000D0000243719AC4200D3F8BD02F07D
:105440008FFC030A3B70631CDBB201379D4203D91A
:105450000234F054E4B2EEE71C00EDE773B5060049
:105460000C000225002819D0002917D0032101A81B
:10547000FFF7DDFF6B469A793F231A400133134350
:105480006A463000937101A92200FFF71BFF051E39
:1054900004D10322E01C01A902F01AFB280076BD0A
:1054A00003785807DA08C00FD20080009B0710432A
:1054B0009B0F1843C0B2704707230B40C908C900AF
:1054C0000B4303707047000070B50400FFF7EAFE5D
:1054D000134DA4006359002B21D0186A002801D075
:1054E00002F0AEFC2B59986E002801D002F0A8FC07
:1054F0002B59D86E002801D002F0A2FC2B59186F4E
:10550000002801D002F09CFC2B59586F002801D0D4
:1055100002F096FC285902F093FC00232B5170BD39
:10552000FC68FF1F0E4B8000C35870B50C00002BA9
:105530000FD09D68002D0CD02B78201D0B706B7840
:105540004B70A97CFFF7B8FF2B7E23726B69E36079
:1055500070BD10220021200002F05AFBF8E7C0467F
:10556000FC68FF1F014B18607047C046F868FF1FBA
:10557000074A03008000825810B5002A06D0D08860
:10558000984203D1012901D1FFF79EFF10BDC0460B
:10559000FC68FF1FF0B5264E95B087000B93BB59F2
:1055A0000500099112200A92002B31D0D888FFF70C
:1055B000A5FB04001420002C2AD0280010A9FFF716
:1055C000B1FFBB591E781D6A002E23D00895FDF748
:1055D000FFFA07000020FDF701FB0790A379E61D05
:1055E000069310AD0CA9089800F0E2FA0EA9280065
:1055F00000F0D7FA0B9B0A990493069B0998029333
:10560000079B0396019300970EAB0CAAFFF77CFE55
:1056100015B0F0BDFDF7DCFA06903000FDF7DEFABC
:10562000E31DA779079310AB06000893DAE7C0469D
:10563000FC68FF1F30B50C4C85002A59030085B06B
:105640000120002A0ED018006946FFF76BFF2B5986
:105650001A78D888054B002A00D1054B6A460721E5
:1056600000F0D9FB05B030BDFC68FF1FA35B021141
:10567000B15B021130B5094C8500295985B0102263
:105680006846253102F024FA2A591121044BD088AA
:105690006A4600F0C0FB05B030BDC046FC68FF1F85
:1056A0004D5C021130B5094C8500295985B0102296
:1056B0006846353102F00CFA2A591121044BD08882
:1056C0006A4600F0A8FB05B030BDC046FC68FF1F6D
:1056D0008B5C0211F7B54D4F86001020F4590D0078
:1056E00002F006FBF3592062186A132200286CD0DE
:1056F000033A29009C6802F0EBF9F3591A780192F9
:10570000002A58D11E6A227D317B944651400122E5
:10571000019F114201D167461740217D91433943D2
:105720002175377B4F40BC4660460027800701D477
:105730004F081740012102208F40227D82433A43C7
:105740002275377B5740BC4660460027400701D48E
:1057500097080F400420227DBF0082433A43227500
:10576000627D002794466046727B42400A4201D126
:1057700067460F400121627D8A433A436275777B19
:105780005740BC4660460027800701D457080F40A9
:105790000220627D7F00824317436775767B00227B
:1057A0007E40760701D4BA080A400426617D920043
:1057B000B1430A4362756A78002A08D06278002AE9
:1057C00005D005220533DA7700221000FEBD042241
:1057D0002979114205D1A17C114202D10533033A46
:1057E000F1E7019A21782C78002A02D10A002100E1
:1057F000140018220429E8D8042CE6D805206043B8
:10580000034A05331218525CDDE7C046FC68FF1FEF
:105810009482021110B50A001121024B00F0FBFA2C
:1058200010BDC046E75C02110B0030B587B001AD7A
:105830002B806B4604001100981D082202F048F9E5
:105840002A000B212000024B00F0E5FA07B030BD22
:105850000F5D021110B50A001121024B00F0DBFAB6
:1058600010BDC046635D021113B50B0011006A46FE
:1058700013706B4604000622581C02F029F96A4690
:1058800008212000014B00F0C6FA13BD835D021110
:1058900010B50A001121024B00F0BDFA10BDC04640
:1058A000D35D02117FB505000B4BAA00D458080048
:1058B000002C0FD0666F237FE28821780396266F35
:1058C0000296E66E0196A46E0094FDF719FC28007E
:1058D000FFF7FAFD7FBDC046FC68FF1F10B517211A
:1058E000FFF7E0FF10BD000070B50A000D00064B89
:1058F0000221040000F08FFA060029782000FFF74B
:10590000D1FF300070BDC046B35C021170B586B0E7
:1059100000236A461370836804001D78681E0A28F5
:1059200059D801A902F094FB060633373B3F4347A1
:105930004B4F5300180000F042F9062312284BD0B9
:1059400000281BD16088FFF7D9F90823002813D05D
:105950004279002A47D1264B1A78072312070BD524
:10596000244B1A680723002A06D01668002E03D09D
:10597000290001AAB04703006A4613706B461B78E2
:105980006088002B2AD1FFF767FC06B070BD1800B5
:1059900000F06CF9D4E7180000F087F9D0E71800A0
:1059A00000F093F9CCE7180000F0ADF9C8E7180053
:1059B00000F0C3F9C4E7180000F0F6F9C0E71800DA
:1059C00000F0F6F9BCE7180000F013FAB8E7180089
:1059D00000F013FAB4E707236A461370694660883B
:1059E000FFF782FFD1E70523012AC5D1024BB8E7B3
:1059F0008967FF1FF468FF1FF868FF1FF8B52C4F79
:105A00008600F35904000D00002B40D0DA88824252
:105A10003DD15A78062A33D11A78002A2ED0012097
:105A200099681A6A097D014206D0157B054203D0A8
:105A300007225A700120F8BD0220014204D0157BD4
:105A4000054201D00922F4E70420014204D0127B70
:105A5000024201D00B22ECE7164B1B68002BE9D069
:105A60005B68002BE6D020009847BB5900215B788B
:105A7000122BDFD12000FFF715FFDBE70E4BECE721
:105A8000112A04D1002900D032252900F2E7002D87
:105A900008D12000FFF732F9002803D01023027943
:105AA0001343037121002800FDF7A8FAC2E7C0469E
:105AB000FC68FF1FF468FF1FF868FF1F70B50E4EEB
:105AC0008500AB590400002B13D01B78002B11D19B
:105AD0000A4B1B68002B04D05B68002B01D0200010
:105AE000984773595B78122B03D100212000FFF7F0
:105AF000D9FE70BD024BECE7FC68FF1FF868FF1F82
:105B0000F468FF1F094B8000C3581020002B0CD0F5
:105B10001A6A002A09D09B68002B06D0127A1B7ED5
:105B2000101C9A4200D9181CC0B27047FC68FF1FB5
:105B300070B503000D0014000220002A30D00029A7
:105B40002ED013700B78081D53704B789370FFF7AD
:105B5000A7FCE070012002212B7A23716B7B0340AC
:105B600063716A7B0A401343042263716E7B1640A3
:105B7000334363716E7BF608F600334363712B7B0E
:105B80000340A371287B014000200B43A371297BB4
:105B90000A401343A3712A7BD208D2001343A37196
:105BA00070BD10B50A0001000120FFF7C1FF10BD54
:105BB00010B50A0001000220FFF7BAFF10BD70B552
:105BC00006000C000220002E30D000292ED0737861
:105BD000201D0B70B3784B70F178FFF76DFC01223C
:105BE0003579257271794B100800134093401040AD
:105BF0000343881010408000C9080343C9000B43C9
:105C00006373B1794B100800134093401040034375
:105C1000881002409200C9081343C9000B43212099
:105C20002373FCF783FE854201D2122070BD22202F
:105C3000257AFCF77BFE8542F7D823781820042BC1
:105C4000F4D86378012BF1D80020EFE7030010B5FA
:105C50000220002909D0002B07D00322481C0A701B
:105C600019000D3201F034FF002010BD03000222A4
:105C7000080010B5002B06D0002904D00E32591CA4
:105C800001F026FF0022100010BD030010B5022015
:105C9000002909D0002B07D00422481C0A701900E3
:105CA0000C3201F015FF002010BD10B5FFF7DEFF2C
:105CB00010BD03000220002906D0002B04D00522CD
:105CC00000200A701B784B70704703000220002BE5
:105CD00008D0002906D05B7800200B70013B082B10
:105CE00000D918307047030010B50220002909D0F0
:105CF000002B07D00622481C0A7019000A3201F056
:105D0000E7FE002010BD10B5FFF7B0FF10BD020088
:105D10000B00022010B500290ED0002A0CD007215C
:105D20001970118859701188090A99701118082280
:105D3000D81C01F0CDFE002010BD03000A00022097
:105D400010B5002B0CD000290AD099785878090298
:105D500001431180901CD91C082201F0B9FE0020DB
:105D600010BD030010B50220002909D0002B07D078
:105D70000822481C0A701900921801F0A9FE0020A0
:105D800010BD02000B00022010B500290BD0002A24
:105D900009D009211970117818185970511C062260
:105DA00001F096FE002010BD10B5FFF75FFF10BD9B
:105DB00002000B00022010B5002A09D0002907D0EC
:105DC0005178197011180622581C01F081FE00202C
:105DD00010BD030010B50220002909D0002B07D008
:105DE0000A22481C0A701900063201F071FE0020D8
:105DF00010BD10B5FFF73AFF10BD02000B000220E6
:105E000010B5002A06D0002904D018005178FFF7F9
:105E100053FB002010BDF0B585B017001E006A4688
:105E200006230500080091819380FEF7C0FC13242F
:105E3000011E02900CD03800B047041E05D1280086
:105E400001A9FEF76FFA041E02D0029801F0C0FE0D
:105E50002800FFF701FA200005B0F0BDF0B50400FE
:105E60008BB0019115000021102202A801F0D0FE94
:105E7000334EA700B85900283CD0C388A34239D17B
:105E80000378002B36D14278062A18D1020001008F
:105E9000553235310C3006ABFFF7A9FA002829D16D
:105EA0002000FFF72FFE020006A902A801F010FE55
:105EB000200002A901F034FE01200BB0F0BD816E7C
:105EC000002917D00B8A112A28D19D420ED10198A2
:105ED0001231093A01F02CFF012807D1BB592000EB
:105EE0009D6EFFF70FFE29000200DEE73221200041
:105EF000FFF7D8FC2000FEF701FF061E1BD0416A09
:105F0000002918D00B8AAB4215D108220198123112
:105F100001F00EFF01280ED1716A0AE09D42E9D11D
:105F200008220198123101F003FF0128E2D1BB5988
:105F3000996E8A7EB9E7200001F002FEBCE7C046F8
:105F4000FC68FF1FF0B56B4D87007E5985B0337834
:105F500002900393002B00D087E0B368346A01936A
:105F60007078062817D101221B7D134202D0217BB5
:105F7000114218D10222134202D0217B114251D189
:105F80000422134203D0237B134200D08BE0019BF9
:105F90005A7DEB5991E007380428F8D802F058F8F8
:105FA000032E42678300B36E002B03D11C2001F047
:105FB0009FFEB066EB599C6E002C1CD01022002175
:105FC000200001F025FE0298FFF79CFD0100200053
:105FD000FFF72DFA01F0C4FE2082200008211230C4
:105FE000FFF725FA0298FFF78DFDA076EB59210007
:105FF000D888FFF70FFC0822EB591CE0B36E002B8A
:1060000005D01A00198AF0881232FFF70DFC02221F
:10601000019B197DEB5911423DD0207B10423AD0B3
:10602000073208E0F488FCF7EBFD01002000FFF7E1
:1060300011FC0A22EB595A70029B9C002A59537892
:10604000073B042B11D8D088FEF758FE00284ED00D
:10605000C3895A08D2182849029B0298CB542B595D
:1060600041180433254801F043FD05B0F0BDFCF7AD
:10607000AFFD03000120834201D100200393EB59BF
:10608000DE88FCF7ABFD039902003000FFF7ECFB64
:10609000019AEB59117D042211420CD0217B11424F
:1060A00009D00B22C7E7F688FCF74CFD0100300051
:1060B000FFF7EEFB6BE7019A527D01210A4204D003
:1060C000607B084201D00C22B5E702210A4204D0CD
:1060D000607B084201D00E22ADE704210A4204D0C1
:1060E000627B0A4201D01022A5E71222A3E7FA221E
:1060F0005200B0E7FC68FF1F0069FF1FBB6402117C
:1061000010B5064B1A780423100018401A4200D02C
:106110000348FFF727FA002010BDC0468967FF1F1C
:106120003446FF1F70B50400FFF7D4FA051E43D1B3
:106130002000FFF77FFA234EA400A0598268937CC9
:10614000DB0708D50321036A1B790B40012B02D121
:10615000017F0B430377431DD97F8B1E022B0DD884
:10616000022900D00121C088FCF7A0FF0421335987
:106170001A7F59700A431A77280070BD01290CD183
:1061800002231022437000210C3001F041FD3059F0
:1061900010213530FFF74BF9EEE70529ECD102234A
:1061A000D118437010220C3001F092FC04233259B4
:1061B000117F0B431377EAE708251828DCD1053D4A
:1061C000DAE7C046FC68FF1FF0B58BB00591438845
:1061D0007E4F9E00F45915000493002C15D101291F
:1061E00002D000200BB0F0BD101D57781678FFF7D5
:1061F00057F9EB68320002932B7A049901930090CF
:106200003B002000FCF71CFFEBE7E388049A934275
:1062100001D00820E6E72378012B00D1D4E0059BCC
:10622000581E092800D9CFE001F012FF05CE0A2937
:10623000CC506C859AB229000498FFF773FFD1E720
:10624000200029001022453001F042FCB9594B785A
:10625000042B02D1013B4B70C3E70B000A0025332E
:1062600035320C310498FFF795F90498FFF702FADC
:106270000522431E9841BB59C0005A70B2E7200066
:1062800029001022553001F023FC049B4F4C9D0047
:10629000295904980A0006AB55320C31FFF77AF9F8
:1062A00029591022453106A801F042FD012808D1E4
:1062B0000498FFF7F7F90590002804D106222B591E
:1062C0005A7005988EE708230593FAE763780C2B3C
:1062D0007AD1E36E002B03D11C2001F009FDE066AA
:1062E000BB59D86E00286FD01022290001F0F0FBB6
:1062F000BB590498DC6EFFF705FC0D22A076BB5954
:106300005A706EE7E06E00285ED063780D2B5BD18B
:106310002B8808220382A91C123001F0D9FBBB593B
:106320009A68517D0222114226D0186A407B1042A1
:1063300022D00C32E4E763780E2B45D1236F002B7B
:1063400003D1162001F0D4FC2067BB59186F002838
:1063500003D01022290001F0BBFB0F22BB59CFE76D
:1063600063780F2B30D1206F0622691C103001F0AA
:10637000AFFBBB599A68517D0422114203D0196AC0
:10638000497B1142D5D100210498FFF78BFA28E709
:10639000636F002B0DD0BB59586F0028F3D010222B
:1063A000290001F095FB0122BB5952425B6F1A6133
:1063B000E9E7142001F09CFCBB5960675B6F002B80
:1063C000E9D126E72978DFE707200BE7FC68FF1F04
:1063D00010B5064C207001F0C3FD06212078FDF7B2
:1063E00091FF0348FEF778FC10BDC0460F69FF1F00
:1063F0007155021100200BB270B50D00834216DA00
:10640000264B187801F05CFB041E0DD00378922B0C
:106410000ED0A02B37D0224B1878FF283AD021007D
:1064200001F016FD002835D180200002684070BDC3
:1064300043780E2B0BD03E2BEDD18378052B12D059
:10644000082BE8D181798088FFF7D8FA08E0154B4E
:1064500082889A42DFD183681878591CFEF7C0FE03
:10646000002817D1D7E7104B1B785B0712D50F4BCD
:106470001B68002B0ED09B68002B0BD0C289811D9E
:1064800080889847ECE7FFF741FAA068002801D020
:1064900001F09EFB200001F0CBFAC5E70F69FF1F5A
:1064A0002D46FF1F182000008967FF1FF868FF1F97
:1064B00010B50078FFF712FA10BD10B50078FFF79D
:1064C000FDFA10BD0C234343084A10B59B185A68C7
:1064D000002A03D0012901D1904710BD9B68002BF1
:1064E000FBD00029F9D19847F7E7C0462C69FF1F78
:1064F00010B5162813D801238340094A946B1C4316
:106500009463506B98435063D46B200098430129E7
:1065100001D120001843D063116B0B43136310BDEE
:1065200000800040F0B500240127154B85B0DA6BE0
:10653000144E03921A6C0192DA64019BE3403B42D1
:1065400017D0039DE5403D400295E5B20299280031
:10655000FFF7B8FF316A736A002908D03900002BB1
:1065600001D0029979402800FFF7C2FF01E0002B1B
:10657000F9D101340C36172CDFD105B0F0BDC0467F
:10658000008000401069FF1F10B5012402002000A8
:10659000162A08D8054B5968D140214204D0186802
:1065A000D0400123184010BD186DF9E7008000406D
:1065B000162807D80122064B8240002903D0D9684B
:1065C0000A43DA607047D9689143D960FAE7C04658
:1065D0000038004030B5162818D8032444430F4B28
:1065E000E25C1B199C785D7801232D1B0135AB40C3
:1065F000013BA340A140DB430C00122807D8084907
:1066000092005218116819402143116030BD054AAB
:1066100011680B4023431360F8E7C046DB82021188
:1066200008F0004014F00040C21F70B5D4B2062339
:10663000092C0BD80125084C9540002908D00021D1
:10664000FFF7C8FF23682B4323600023180070BDA9
:106650002368AB43F8E7C04600380040F0B5162881
:1066600026D8214B1B185B78022B21D103244443ED
:106670001E4A1F4EA35C1219947801221500854012
:10668000B76B013CE4B23D43A240B563194C1228FC
:1066900015D89B0000290CD117495B1899680A434B
:1066A0009A600123205C154A834011680B431360F4
:1066B000F0BD11495B18996891439960F1E70E4B61
:1066C00000290DD159690A435A61225C1328E8D088
:1066D0000123203A93400A49086803430B60E7E727
:1066E000596991435961F0E71069FF1FDB8202117C
:1066F000008000402083021100F00040A0F0004024
:10670000A4F00040F8B500241B4E1C4D1C4B1B5D33
:10671000012B1FD1184A9269E2401A420BD0012284
:10672000AA5693402200143AD2B2022A09D8154937
:106730004A6913434B6101340C360235172CE5D1FD
:10674000F8BD0022AA560F499200521891680B43D7
:106750009360F0E7022BEED1E7B23800FFF714FFA9
:1067600001235840C1B23800FFF778FF3800FFF727
:106770000BFF7077DFE7C0461069FF1FAD82021183
:106780001169FF1F00F00040012202388240054BD2
:10679000002903D059690A435A61704759699143E6
:1067A0005961FAE70038004070B504000D0005207B
:1067B000162C1AD800212000FFF7FAFEA31E012B89
:1067C00003D801212000FFF7DFFF00212000FFF7A1
:1067D0002BFF01220A49A2400A4B4868012D05D12E
:1067E00002431B194A605D70002070BD90434860F1
:1067F00002211C196170996991439961F4E7C046BF
:10680000008000401069FF1F10B516280AD8012229
:10681000074B8240002906D019680A431A600121FB
:10682000FFF7C2FF10BD196891431960F7E7C04632
:106830000080004070B505000520162D17D80C23E8
:1068400000246B430A4A21009B181C70094B280046
:106850005B195C70FFF7A8FF0123AB4020000649DD
:106860000A681A430A6005490A689A430A6070BDBB
:106870002C69FF1F1069FF1F3480004030800040EA
:1068800070B504000E00FF2813D003250540FFF764
:10689000D1FF084AA3089B009B183F22ED00AA40A5
:1068A000AE40196820009143314319600121FFF780
:1068B0007FFE70BD18380040F8B505000520162D84
:1068C00025D80C246C43124BE4186368002B03D1C9
:1068D000A3680D30002B1AD0022201270D4B002196
:1068E0005B195A7028002770FFF75EFF63681E1E51
:1068F00008D0A3683E00002B04D02800FFF744FE18
:106900004640F6B228003100FFF7F2FD0020F8BD46
:106910002C69FF1F1069FF1FF7B5C420FF222B4B06
:1069200080001958002491437F3A0A431A5080226C
:10693000274F5202274E1A60274B1D5D002D21D094
:10694000A31E012B03D80121E0B2FFF71DFF012D8B
:1069500018D11F4B9B69E3402B4213D0E3B21800C0
:106960000193FFF711FE01000198FFF74DFFE3B21D
:10697000143B022B1DD801217156184A8D405369D2
:10698000AB4353613B7F002B0DD0E5B22800FFF7EE
:1069900093FF2800FFF7F8FD7B7F0100834202D0C0
:1069A0002800FFF78FFD01340C370236172CC3D1B6
:1069B000F7BD012100237156F3568D40074A9B0015
:1069C0009B189A68AA439A60DCE7C04600E100E0A1
:1069D0001069FF1FAD8202111169FF1F00F0004016
:1069E00010B504000520162C0CD801212000FFF75B
:1069F000DBFE0123044A002011194B70A34091696A
:106A00000B43936110BDC0461069FF1F70B50E00A7
:106A100015000400FFF70EFF0C236343094A200012
:106A20009B189D605E60FFF747FFF021064B074A09
:106A30008900051E5A5002D02000FFF7FBFE2800F7
:106A400070BDC0462C69FF1F0000FF1F25650211A5
:106A500070B5134D07202C78002C1FD198222100EF
:106A60005200280001F0CCF90123C420FF222B7032
:106A70000C4B80001C635C630B4B1C605C600B4B1D
:106A8000195891437F3A0A431A50802252021A60E1
:106A90000D20074A074901F083F8200070BDC04669
:106AA0001069FF1F00800040A0F0004000E100E0FE
:106AB0001969021105670211030010B50620072BA2
:106AC00009D8054A137001F05BFAD7210020034B67
:106AD000034A89005A5010BD5C46FF1F0000FF1F8B
:106AE000151BFF1F70B51D0002240C2910D8094A80
:106AF000CA40D2070CD5FBF725FF041E08D1059A22
:106B000004992800FBF73AFFFCF7A8FDFFF7F8FA15
:106B1000200070BD1210000030B50D7802232C004B
:106B20009C43184201D02B431C0008252300AB4393
:106B3000284201D02B00234320241D00A5432042DE
:106B400001D01C4325002A230D70184204D011786F
:106B50001E3B0B43137030BD0028FCD10C21137871
:106B60008B43F7E7F8B51D0006AB1B88140007AA96
:106B70000E000B201778002B27D10A78022A49D162
:106B80004A68507811780002244A08438018042883
:106B900040D801F05DFA03121D1B2300F06801F0DC
:106BA0004FF8021CC0B2B84200D93A1CD2B2200041
:106BB000F1682A8000F08CFF06E00222F3681B884F
:106BC0002A8023701B0A63700020F8BD0622EEE7BE
:106BD00001232B80F3681B782370F5E7F368002B03
:106BE00016D008222A801A8822701A88120A627027
:106BF0005A88A2705A88120AE2709A8822719A887A
:106C0000120A6271DA88A271DB881B0AE371DBE782
:106C10002B80D9E701202B80D7E7C04600D6FFFFA5
:106C2000F7B516000A781D0008AB1F880C00012379
:106C3000022A18D14A685078117800022B4A08437A
:106C4000801803280FD801F003FA02254439E068C0
:106C500000F0F6FFC0B20723B84204D37B190193BA
:106C6000152B02DD0D231800FEBDE0682A0031005F
:106C7000C01900F02DFF6B4600209B88E268D054BD
:106C80001B4B1B68834203D01B68834200D098478C
:106C90000023E8E70B23002FE5D1022DE2D1737822
:106CA00032781B021343E2681380114B1B68002BE0
:106CB000EED01B68002BEBD00120E8E70B23002F60
:106CC000D1D1062DCED12A003100E06800F000FFBE
:106CD000DEE70B23002FC6D1012DC3D132787533E7
:106CE000012AC0D8E3681A70D2E7C04600D6FFFF79
:106CF0001C6BFF1F70B50C001500072837D801F07A
:106D0000A7F9041436361B36242E182015290BD863
:106D1000184E16220021300000F07AFF22002900D0
:106D2000300000F0D5FE002070BD18200229FBD1F4
:106D30001288114B1A80F6E718200829F4D10A00AE
:106D40000E48290000F09CFFEDE718200129EBD147
:106D50000B4B10780B49DA69FFF7DEFEE3E71820EA
:106D60000129E1D1064B10780749DA6BF4E70220DC
:106D7000DAE7C046046BFF1FDA46FF1FD046FF1F4D
:106D80006046FF1F8846FF1FA846FF1F030010B57F
:106D90000020DB0704D50721024A034800F08CF8E5
:106DA00010BDC046388302116046FF1F054A03002C
:106DB0001068002803D082889A4201D18068704709
:106DC0000068F6E7206DFF1F0A88030008009A425A
:106DD00004D08A8804309A4200D000207047000016
:106DE000F8B5F82200230D4F0D4E79680500424397
:106DF0003370994200D07B600A4C0021200000F0E3
:106E000007FF00231A007C60AB4202D100203370E0
:106E1000F8BD01332280DBB2F834F5E7206EFF1FA6
:106E20001C6EFF1F246DFF1F73B56B46019006009B
:106E3000684615001980FCF743FF041E11D1002D90
:106E40000FD07689002E11D00C2000F051FF0028C1
:106E50000ED0084A0460136886808560002B02D13A
:106E60001060200076BD1A001B68F7E70224F8E7DF
:106E70001324F6E7206DFF1F012100220A4B10B5F5
:106E800049420A4C198099809A719A70084B207077
:106E9000012019805A60FFF7A3FF2078FCF76EFFEE
:106EA0000448FDF719FF10BD246BFF1F286EFF1F5C
:106EB000206EFF1F656F0211022310B5002802D05B
:106EC000FFF7B2FF0300180010BD0000030010B56B
:106ED0000020DB0704D50421024A0348FFF7A4FF82
:106EE00010BDC0464C830211E046FF1FF0B50E26D0
:106EF00087B003930CAB1F8802ABF618050008009F
:106F000031000292FDF75EF804000120002C0FD042
:106F10003088FFF74BFF03000E20002B08D05E687F
:106F2000002E05D021002800039B029A0097B0474D
:106F300007B0F0BD0A4B10B5984207D101220023DB
:106F400052420A808B708A808B7110BDFFF73CFF24
:106F50000028FAD001235B42038000238370F4E70A
:106F6000FFFF0000F8B5050001290AD1134E0024E7
:106F70003388F827AB4219D028001149FFF7DAFF10
:106F800006E0022904D10139FDF724FF0028EDD0E5
:106F9000F8BD3B0063437268D018D35A002B09D068
:106FA0003A00002100F034FE0134E4B2054B1B78B6
:106FB000A342EED801235B423380DDE7206EFF1F42
:106FC000246BFF1F1C6EFF1F10B5FFF7FDFE0300B3
:106FD0000020834200D0987810BD0000F0B589B041
:106FE0001C000EAB80CB03901E8810AB1B78049264
:106FF00002930B7A0D00DB0616D42B780593022B37
:1070000024D00498FFF7D2FE002812D003689C46D3
:10701000002B0ED0029B2200019329003B00644606
:1070200003980096A04705E00498FFF7BFFE0028EC
:1070300002D10E2009B0F0BD8368002BF9D00A22DE
:107040002900039898470028D7D0F3E76B68587851
:107050001A786B4B000210439842D2D8043B9842F6
:1070600010D2684B984242D015D8674BC0180128FF
:10707000C7D80B20002EDDD1EB681A7859683A800A
:10708000200028E0614BC018032800D979E000F007
:10709000DFFF846A789E5E4B9842B2D10B20002EAF
:1070A000C8D101233B80EB6831001B7823706889CD
:1070B000013080B2FCF786FF3A88031E0ED00178BB
:1070C00002328A183A80428962704289120AA2709A
:1070D00059680278E01C00F0FBFC06E004323A80BC
:1070E00031000422601C00F093FD0020A2E70B2079
:1070F000002E9FD1EB6807A91E8804233B80330A2A
:10710000300026706370FCF75DFF051E28D004ABCD
:107110009A890E2304A95B183E49C668FCF7C6FF8E
:1071200000280BD12B783C486A680599FBF77CFB5B
:10713000002803D1012304AA5B42D3813278022ABA
:1071400006D17168201D00F0C3FC3B8802333B80F0
:107150000E2304AA9B181B88A3701B0AE370C4E7C4
:1071600004ABDE81F4E70B20002E00D062E7E96873
:107170000398FFF729FF02233B802070000A60700C
:10718000B3E70B20002E00D054E70222EB681B88E7
:107190003A8023701B0A6370A7E7E86800F050FD8F
:1071A000C2B203000720B24200D243E70DD00299D9
:1071B000DBB27118994202DB921BD3B20293029B9D
:1071C000E9681A003B8089195AE70023F6E70B208B
:1071D000002E00D02EE70722EB683A801A78227042
:1071E0005A7862705A88A2705A88120AE2701A7924
:1071F0002271DA886271DB881B0AA37175E7C046C9
:10720000042900000228000000D8FFFFFFD6FFFF7E
:1072100003280000FFFF00007C820211F0B58DB052
:107220006B460020089120229B5E83423DDAA64BEC
:10723000187800F045FC071E32D00378B02B2CD113
:107240000079023816281FD800F062FC17001E00D3
:107250001E001E0031001E0096001E001D011E00B3
:1072600052011E0073011E00CD011E0050021E00BF
:107270001E001E008E021E00E302944B94491B88E0
:1072800078880B80FBF710F83800FCF781FF914BF2
:107290001B68002B01D038009847380000F0C8FB6D
:1072A0008020089B0002434018000DB0F0BDF6227C
:1072B0000021874800F0ACFC0BAA3B7B7989388918
:1072C00000923A000D32FCF795FD0400804B1B78CC
:1072D000002C3FD146E0804B788805937F4B4100DE
:1072E000CB5A0BAE073BDBB23288029300230193EB
:1072F0007B4B210006930093059BFFF76FFE744DB7
:10730000002810D1069B3A8A1B889A420BD138007C
:107310000599123000F00CFD002804D02B7862890A
:107320009B00EB185A80162306A81B1832882000F1
:107330007989FCF7BBFE2B7804009A00AA185188C3
:107340000029C3D00133DBB22B70002807D006A977
:10735000C98A9180634A12889A42BCD802E001210E
:1073600049429180002B04D059497888FAF7D0FF20
:107370008AE73E890A2479E000253E89574B069327
:107380007B88069A5B009B5A033B9D4202DB002DE3
:10739000F0D05BE0162206A812183B7B7989009298
:1073A0003A0030000D32FCF725FD0590002858D03A
:1073B0004689017A7888FCF7E7FC041E44D1464BE5
:1073C00078880793069B4100C95A454B0439C9B2D6
:1073D00006AAD28A06930291019400930599079B0D
:1073E000FFF7FCFD041E2FD1069B39491A88931C18
:1073F000002D26D14B807988384B4900CB5A511942
:10740000033B8B4220DD059B31485B8941190B71A1
:10741000A91C0135C9B2EDB2059145191B0A2B71A2
:10742000059B2D490433181800F052FB2C4B059A8C
:107430001B88D318DDB22C4B9E4205D00136B6B264
:107440009CE749889942D6D0002D0CD0204C2800CA
:10745000618800F095FC207021007888FAF768FFB9
:1074600012E7059CF0E7002C00D183E77B78142B12
:1074700000D109E716493B794E800B700C71788872
:10748000FAF708FF00E7162406ABE4182100388954
:10749000FCF798FD011E00D1B7E1788822880F4CD7
:1074A00045002C5B0A4D013CE4B2029400240F4BD2
:1074B00001940095FFF792FD041E00D014E129000D
:1074C0007888FAF745FFDFE6286EFF1FCC45FF1FDF
:1074D0002C6BFF1F206BFF1F266CFF1F5C67FF1FBD
:1074E0001C6DFF1FCA45FF1FFFFF00002E6BFF1F13
:1074F000162406ABE41821003889FCF763FD011E51
:1075000000D182E178882288AE4C45002C5BAE4DDC
:10751000013CE4B202947C89AC4B01940095FFF7E6
:107520005DFD041E00D0DFE029007888FAF71AFF1D
:10753000AAE60025A44B1D803B00FE331B78A24A1F
:1075400078880792AB4208D99E4B12880693069919
:1075500043005B5A013B9A4203DB0799FAF70CFFA1
:1075600092E616246B00FB18059306ABE418059B06
:1075700021001889FCF726FD011E03D1059B01247B
:107580001E8973E77888924B2288069C09934300F2
:107590001B5B904E013BDBB20293002300960193EC
:1075A000099BFFF71BFD041E02D0059B1E895DE7AA
:1075B0007B88069A5B009B5A079A108832881218BB
:1075C000934202DC1B1A013B33807F4C023032882D
:1075D0000999001900F07CFA2388328801359B183C
:1075E0002380EDB2A8E70BAA3B7B7989388900920A
:1075F0003A000D32FCF7FEFB00250590059B002BA1
:1076000004D10A24002D00D16EE060E0059B78884B
:10761000197AFCF7B9FB0100041E63D1694C6C4B6D
:10762000788806940993069B4400E45A694B063C0B
:10763000E4B20BAE3288079302940191009305994E
:10764000099BFFF7CBFC041E4CD1079B5E491B88AE
:107650001A1D002D30D14A80059B5B4C5A89631955
:107660001A716B1C9BB2E318120A1A71162306A832
:1076700032881B1879890598FCF718FDFF21AA1C90
:107680002E1D03350B00059092B2B6B2ADB20028A4
:1076900003D006ABDB8AD9B21B0AA2186519117197
:1076A0002B714C4D301D2A884949201800F010FAE2
:1076B0002B88F618B5B2A1E74988914207D17A889C
:1076C00006995200525AEB18053A9A42C4DC3E4CD5
:1076D0002800618800F06CFB207021007888FAF7A0
:1076E00055FED1E5002DF2D13E89BFE6162606AB48
:1076F000F61831003889FCF765FC3D000400FF35C1
:1077000000282DD0037A9B060CD400227B8939896E
:10771000788800923A000C32FFF7E8FB041E10D084
:107720003E8915E03088FFF741FB00281AD08368B6
:10773000002B17D02100122278889847041EE4D02D
:10774000EEE7AB78002B02D17888FAF72FFE0026FF
:10775000AB78002B00D097E5002C00D194E585E6AE
:107760000124DDE70E24DBE7162506ABED18290022
:107770003889FCF727FC041E47D0037A9B0611D4F6
:10778000154A7B881188994203D01448814207D159
:107790001380134BF8261D780023D9B2A94221D3B8
:1077A0000924A1E72888FFF701FB00282FD0836870
:1077B000002B2CD02100122278889847041EDFD09D
:1077C00092E7C0465C67FF1F2C6BFF1F2E6BFF1FED
:1077D000266CFF1F1C6DFF1F206EFF1FFFFF0000A8
:1077E0001C6EFF1F31005943546801336018615A01
:1077F0000029D2D13C0008342100F82200F068F9B9
:1078000021007888FAF7DAFD3EE501246CE70E24C2
:107810006AE71D4B1A887B889A4231D07888FAF73C
:10782000D7FD31E5F823059851684343CD18C95A6F
:1078300000291FD03B7A012B0BD16C88AB8878884C
:10784000AA1D0094FFF752FB041E02D000233B72D6
:107850002E88F8220021280000F0DAF900232B807E
:10786000059B0133DBB20593084B05991B78064A4B
:107870008B42D7D801235B421380002CCED0F5E594
:10788000002634000596EFE7206EFF1F1C6EFF1FD9
:1078900070B504000E001500FFF796FA031E08D11C
:1078A00031000548FFF790FA03001120002B02D0A9
:1078B0001C8000209D7070BDFFFF0000F8B50B4FCD
:1078C00006003B780D001400FF2B0ED00A2000F0BC
:1078D00047F9011E09D0B1230380002346800371BC
:1078E000C5800481387800F0B3FAF8BD2147FF1F46
:1078F000F7B50F0008A90600088809A90B24098814
:10790000002821D10234022B1ED1557813782D0284
:107910001D432B008B4301937334002B14D1FB6860
:10792000300019000093FFF74FFB019C85420BD0FC
:107930002A0030000099FFF7ABFF041E04D12A0093
:1079400030007989FFF7BAFF2000FEBDF0B50E7850
:1079500085B003900AA805880120022E0DD14C683D
:107960002778647824023C43054FBC4205D1039834
:10797000DBB201960095FFF7BBFF05B0F0BDC04636
:107980000229000010B504000C4800F0E1F80C4892
:10799000A16B00F0DDF80B48E16B00F0D9F80A4864
:1079A000216C00F0D5F8094B0948196800F0D0F8AF
:1079B000084B1B68002B00D09847FEE7928102110C
:1079C000A8810211B7810211C681021104ED00E005
:1079D000D58102112C6EFF1F002307B501A801936A
:1079E000FFF7D0FF044A0548002110B5121A00F035
:1079F0000FF9F8F771FFFEE7306EFF1F2447FF1FF6
:107A000001B40248844601BC604700BF5118FF1F03
:107A100001B40248844601BC604700BFAD39FF1F76
:107A200001B40248844601BC604700BF75A900004C
:107A300001B40248844601BC604700BF434D0100C9
:107A400001B40248844601BC604700BFC53F000046
:107A500001B40248844601BC604700BF55220000C3
:107A600001B40248844601BC604700BF21240000E5
:107A700001B40248844601BC604700BFB938FF1F0B
:107A800001B40248844601BC604700BF01240000E5
:107A900001B40248844601BC604700BF595201004E
:107AA00001B40248844601BC604700BF055E000087
:107AB00001B40248844601BC604700BF0189000050
:107AC00001B40248844601BC604700BFF54E010086
:107AD00001B40248844601BC604700BFE94C010084
:107AE00001B40248844601BC604700BFB14E0000AB
:107AF00001B40248844601BC604700BFA9460100AA
:107B000001B40248844601BC604700BFE54800005C
:107B100001B40248844601BC604700BF093EFF1F14
:107B200001B40248844601BC604700BF311B00001D
:107B300001B40248844601BC604700BFEDA50000C7
:107B400001B40248844601BC604700BF091B000025
:107B500001B40248844601BC604700BFE53A010019
:107B600001B40248844601BC604700BF1D4D0100BE
:107B700001B40248844601BC604700BF11470100C0
:107B800001B40248844601BC604700BF456B010058
:107B900001B40248844601BC604700BFA93BFF1FF7
:107BA00001B40248844601BC604700BFD134FF1FC6
:107BB00001B40248844601BC604700BFC935FF1FBD
:107BC00001B40248844601BC604700BFA532FF1FD4
:107BD00001B40248844601BC604700BFD949010096
:107BE00001B40248844601BC604700BF313BFF1F1F
:107BF00001B40248844601BC604700BF7D18FF1FE6
:107C000001B40248844601BC604700BFD1A5000012
:107C100001B40248844601BC604700BF154D010015
:107C200001B40248844601BC604700BF3134FF1FE5
:107C300001B40248844601BC604700BF3D18000003
:107C400001B40248844601BC604700BFDD52010018
:107C500001B40248844601BC604700BFF30E000037
:107C600001B40248844601BC604700BFE1AC00009B
:107C700001B40248844601BC604700BF613AFF1F5F
:107C800001B40248844601BC604700BF810E000079
:107C900001B40248844601BC604700BF2146010090
:107CA00001B40248844601BC604700BFE53CFF1FA9
:107CB00001B40248844601BC604700BFED4A0100A0
:107CC00001B40248844601BC604700BF1D3BFF1F52
:107CD00001B40248844601BC604700BF6DBC00008F
:107CE00001B40248844601BC604700BFE1170000B0
:107CF00001B40248844601BC604700BF3D4B01000F
:107D000001B40248844601BC604700BF8B520100A9
:107D100001B40248844601BC604700BFD91B000083
:107D200001B40248844601BC604700BF5D170000F3
:107D300001B40248844601BC604700BFCD4C01003D
:107D400001B40248844601BC604700BF45510100B0
:107D500001B40248844601BC604700BF017F0000B7
:107D600001B40248844601BC604700BF29510100AC
:107D700001B40248844601BC604700BFE93BFF1FD5
:107D800001B40248844601BC604700BF350E0000C4
:107D900001B40248844601BC604700BFC521000011
:107DA00001B40248844601BC604700BFE13DFF1FAB
:107DB00001B40248844601BC604700BF090E0000C0
:107DC00001B40248844601BC604700BFB54C0100C5
:107DD00001B40248844601BC604700BF9DA9000071
:107DE00001B40248844601BC604700BF8D12000008
:107DF00001B40248844601BC604700BF0D52010037
:107E000001B40248844601BC604700BFB70E0000C1
:107E100001B40248844601BC604700BF291C000031
:107E200001B40248844601BC604700BF5937FF1FB8
:107E300001B40248844601BC604700BFA54F010061
:107E400001B40248844601BC604700BF014C0100F8
:107E500001B40248844601BC604700BF594F01008D
:107E600001B40248844601BC604700BF0936FF1FC9
:107E700001B40248844601BC604700BF090E0000FF
:107E800001B40248844601BC604700BFB352010000
:107E900001B40248844601BC604700BFC95C0100D0
:107EA00001B40248844601BC604700BFD13CFF1FBB
:107EB00001B40248844601BC604700BF851F000032
:107EC00001B40248844601BC604700BF252600007B
:107ED00001B40248844601BC604700BFC9A9000044
:107EE00001B40248844601BC604700BF1D4B01003D
:107EF00001B40248844601BC604700BF4D1F00002A
:107F000001B40248844601BC604700BF8934FF1FAA
:107F100001B40248844601BC604700BF51470100DC
:107F200001B40248844601BC604700BF056A0000F6
:107F300001B40248844601BC604700BFE928000044
:107F400001B40248844601BC604700BF79180000B4
:107F500001B40248844601BC604700BF553CFF1F86
:107F600001B40248844601BC604700BFC926000036
:107F700001B40248844601BC604700BFADAE0000BA
:107F800001B40248844601BC604700BF151BFF1FB7
:107F900001B40248844601BC604700BF355500006B
:107FA00001B40248844601BC604700BF693BFF1F23
:107FB00001B40248844601BC604700BF85520100FD
:107FC00001B40248844601BC604700BF691F00003D
:107FD00001B40248844601BC604700BF6936FF1FF8
:107FE00001B40248844601BC604700BF4934FF1F0A
:107FF00001B40248844601BC604700BF512500001F
:1080000001B40248844601BC604700BFF94C01003E
:1080100001B40248844601BC604700BFC94A010060
:1080200001B40248844601BC604700BFC51D000082
:1080300001B40248844601BC604700BF45500000BF
:1080400001B40248844601BC604700BF55490100A5
:1080500001B40248844601BC604700BFF53DFF1FE4
:1080600001B40248844601BC604700BF5932FF1F7B
:1080700000020103020303030403050206020702D0
:10808000080209000A030B030C020D020E030F0382
:10809000100311031303140315001600790C0211C9
:1080A000AD0C02110000000002000000B2800211BD
:1080B000192A0F180A000000F1590000FD240000E1
:1080C00041460100E1430211F563021169380211D2
:1080D000E5410211251D02111D720211F119021153
:1080E000410E0211AD0E0211000000001E0E000034
:1080F00002000000FC800211F4FFF3FFF0FF00001B
:1081000005100211000000000000000054757961A4
:108110000056302E36003030303100676974687593
:10812000622E636F6D2F707676780042544830313E
:10813000000000000200000048810211292A282ABC
:10814000272A262A252A242A0A180000E2040000E9
:108150007102000078EC000074400000102700005D
:1081600060F00000000000001F501D000206B40077
:10817000303132333435363738394142434445465D
:10818000005048592B36325858504C5553303530E2
:1081900034005B48617264206661756C74206861AC
:1081A0006E646C65725D0A004C522020203D2030C8
:1081B00078253038780A0050432020203D20307840
:1081C000253038780A0050535220203D2030782541
:1081D0003038780A0049435352203D20307825300A
:1081E00038780A00352102118921021100000000AF
:1081F00002000000FC8102116F2A6E2A1A18FB345B
:108200009B5F800000800010000000000000000064
:108210006B240211F53A02118F240211FD3E021166
:1082200013250211D33E021189250211A93E021124
:10823000DB25021171400211432602117140021127
:10824000752602112B40021189250211613E02118F
:108250000126021109400211000000000000000088
:10826000E726021109400211492702110D3B0211B4
:10827000052A042A012A002A0229032801280028A5
:1082800001180018000000000000000000000000BD
:108290000000008701010201020101020102030343
:1082A00004010301010101010303020103000D00A8
:1082B0000E001000110013001401070108010A014B
:1082C0000B011C011D02040205020702080219022B
:1082D0001A021C021D03010302031700020100051C
:1082E00004000807000B0A001716001D1C010201FC
:1082F000010504010E0D01111001141301171601DF
:108300001A19020201020B0A020E0D0211100214C8
:1083100013021716030504030807030B0A030E0DC7
:108320000001020307090A0B0E0F1011121417188F
:10833000191A1B1F20212200656B0211216C0211EA
:108340000000000002000000828202110000000014
:108350004D7902110000000002000000808202112D
:020000041FFFDC
:1000000000000000D50D0211B8800211B480021169
:100010003064FF1F0000000000000000000000002E
:1000200000000000000000000000000000000000D0
:1000300000000000000000000000000000000000C0
:1000400000000000000000000000000000000000B0
:1000500000000000000000000000000000000000A0
:100060000000000000000000000000000000000090
:100070000000000000000000000000000000000080
:100080000000000000000000000000000000000070
:100090000000000000000000000000000000000060
:1000A0000000000000000000000000000000000050
:1000B0000000000000000000000000000000000040
:1000C0000000000000000000000000000000000030
:1000D0000000000000000000000000000000000020
:1000E0000000000000000000000000000000000010
:1000F0000000000000000000000000000000000000
:1001000000000000000000000000000000000000EF
:1001100000000000000000000000000000000000DF
:1001200000000000000000000000000000000000CF
:1001300000000000000000000000000000000000BF
:1001400000000000000000000000000000000000AF
:10015000000000000000000000000000000000009F
:10016000000000000000000000000000000000008F
:10017000000000000000000000000000000000007F
:10018000000000000000000000000000000000006F
:100190002D36FF1F1D35FF1FC16601000000000046
:1001A000000000000000000000000000000000004F
:1001B000000000000000000000000000000000003F
:1001C000000000000000000000000000000000002F
:1001D000000000000000000000000000000000001F
:1001E000000000000000000000000000000000000F
:1001F00000000000000000000000000000000000FF
:1002000000000000000000000000000000000000EE
:1002100000000000000000000000000000000000DE
:1002200000000000000000000000000000000000CE
:1002300000000000000000000000000000000000BE
:1002400000000000000000000000000000000000AE
:10025000000000000000000000000000000000009E
:10026000000000000000000000000000000000008E
:10027000000000000000000000000000000000007E
:10028000000000000000000000000000000000006E
:10029000000000000000000000000000000000005E
:1002A000000000000000000000000000000000004E
:1002B000000000000000000000000000000000003E
:1002C000000000000000000000000000000000002E
:1002D000000000000000000000000000000000001E
:1002E000000000000000000000000000000000000E
:1002F00000000000000000000000000000000000FE
:1003000000000000000000000000000000000000ED
:1003100000000000000000000000000000000000DD
:1003200000000000000000000000000000000000CD
:1003300000000000000000000000000000000000BD
:1003400000000000000000000000000000000000AD
:10035000000000000000000000000000000000009D
:10036000000000000000000000000000000000008D
:10037000D979021100000000000000000000000018
:10038000000000000000000000000000000000006D
:10039000000000000000000000000000000000005D
:1003A000000000000000000000000000951AFF1F80
:1003B000000000000000000000000000000000003D
:1003C000000000000000000000000000000000002D
:1003D000000000000000000000000000000000001D
:1003E000000000000000000000000000000000000D
:1003F00000000000000000000000000000000000FD
:081838003072FF1F4118FF1F71
:10184000024981F3088802F03BFB00003072FF1F61
:1018500010B502F015FD072804D0122808D0022880
:1018600008D010BD044A0420136B01331363F8E75A
:101870000220F6E71420F4E70468FF1FF8B507001C
:101880000C0026002500503630785135002804D150
:101890000300287058342370F8BD2978CA00481E08
:1018A0008141A3183800A25C5B68C9B2FFF7D0FF82
:1018B00000280DD12B78DA00A218013350602B706C
:1018C0003378044A013B3370136A01331362D8E75B
:1018D0000123DFE70468FF1F5C234343074910B57A
:1018E000C9180B0058331B78012B05D1FFF7C6FF31
:1018F000034A936A0133936210BDC0463868FF1FE4
:101900000468FF1F10B502F05BFB064A01211300BB
:1019100010CB4942D967044B136002F0E1FA200072
:1019200010BDC04600E100E01000100010B504003A
:1019300002F046FB024B1C6002F0D2FA10BDC0461A
:1019400000E100E010B5040002F03AFB4021094A32
:10195000200013688B43136002F032FC01F048FE54
:101960000022054B01201A60044B04321A6002F079
:1019700057FAFEE71CF00040C4F00040C0F0004001
:10198000431E5A425341A022F0B5D2015B4213409C
:10199000154D164A40019B182A18127E8BB00191F2
:1019A000002A1BD01A000832D46F0022E6B206AF1C
:1019B000E4B294420EDC2818C369002B08D00199C8
:1019C00002AA117106AA049202AA167303A89847E4
:1019D0000BB0F0BD1978B9540132EAE71A7D1A78D4
:1019E00006AB01261A70E6E7C46AFF1F00400040FC
:1019F000F0B5254B04004001C25C85B0002A2BD015
:101A00001A18117E002927D0917E002924D011793F
:101A1000022921D11689D788D168F51BADB22A1CBD
:101A2000102D00D9102292B2BE4217D118180123EE
:101A300003710023C269C38003819A4206D06846BD
:101A4000032103730171029301A890470820002C21
:101A500000D0192001F018FD05B0F0BD013C654231
:101A60006C41A0256442ED012C40084D1B186419FF
:101A7000074D0633013A92B2AA42EDD01888461CAF
:101A80001E80085C2070F5E7C46AFF1F004000401C
:101A9000FFFF00000F220E4B10B59868104002386F
:101AA0000A280BD802F0A6F90D0A0B0A0A110A0A35
:101AB0000A0A060002210020FFF762FF10BD012183
:101AC000F9E70020FFF794FFF8E7DB6FF6E7C04681
:101AD000004000400F220E4B10B5986810400238AD
:101AE0000A280BD802F086F90E0A0B0A0A120A0A13
:101AF0000A0A060002210120FFF742FF10BD012162
:101B00000800F9E70120FFF773FFF7E7DB6FF5E760
:101B10000090004013B5334C2378072B3DD8324B4F
:101B20001A78324B002A39D18022196852020A43AE
:101B30001A60252002F018F820232D4A11680B4363
:101B4000802113606B460422C905086807331042E0
:101B500028D080210422C905C86810422ED08021D7
:101B60002020C905CA688243CA6014221A701A78F4
:101B7000002A2FD18021C905C86820320243CA60DB
:101B800014221A701A78002A28D11A4B1A7D22784A
:101B90005A601D221A705932DA6013BD1A6816494C
:101BA0000A40C5E7086802430A6014221A701A78CE
:101BB000002ACED01A78013AD2B2F7E7C8680243B9
:101BC000CA6014221A7019784A1ED2B21A700029FB
:101BD000F9D1C4E71A78013AD2B2C7E71A78013AC4
:101BE000D2B2CEE75C46FF1F2447FF1F3CF0004007
:101BF0005446FF1F00200040FFFFFEFF564B70B50C
:101C00001B68012B03D1554A936D0133936502F094
:101C100097F9534B534A1860534B544C1A600123A5
:101C2000534A1360534A13602378002B06D00622D0
:101C30005149524802F0DCF900232370504A514BBD
:101C400010681B78C1B2002B0ED14F4CC0B2237864
:101C50005BB2002B4FDB237824785BB264B21B04A9
:101C600024021B191B1813600B1C50294ED950233A
:101C7000464A47491078DBB2FF2202284BD1086858
:101C8000444C454D267890432A78964254D9227880
:101C900024782E78023B5D10A31B6B435201D31AAC
:101CA00010335B111843086002F0F2FA031F012B96
:101CB00045D83A4B1B78002B06D0394B1B78002BAC
:101CC00002D0002002F02CFAA122364B9200997823
:101CD000354B4A431B689B18832292009B181B7844
:101CE000033B012B03D8AF20400002F049FA012248
:101CF0002E4BDA8270BD237824785BB264B2FF3356
:101D0000FF341B0424021B190138ABE7CAB2022AB4
:101D1000AED20223ACE70868254C264D26789043C6
:101D20002A78964208D9227824782D78023B5B10D5
:101D3000641B63435201B2E72378DBB2B2E70228A7
:101D4000D5D11D4B1B78013B022B03D91B4B1B78B4
:101D5000022BCCD16C20C8E79809FF1FFC0FFF1F96
:101D60003C67FF1FFF3F0000141003404067FF1F48
:101D70000C10034000100340D50BFF1F7211FF1F12
:101D8000B40003408C09FF1F680AFF1F490AFF1FA8
:101D900094000340460AFF1F470AFF1FF908FF1F70
:101DA0002209FF1F300DFF1F3409FF1FBC0BFF1F4F
:101DB000440AFF1F450AFF1F1C09FF1F2309FF1FBD
:101DC00010B502F0CDFA0022014B1A8010BDC046BA
:101DD0003867FF1F10B502F0EBF8A121054A890012
:101DE0009478054A61431268044B5218528C1A8049
:101DF00010BDC046300DFF1F3409FF1F3867FF1F9D
:101E000010B50D4B0D4A9978A1239B004B431268E6
:101E1000D218531DD97F0A4B1B88994209D2441C02
:101E200007D0C82805D0D2695B1A5A43054B5343E3
:101E3000C01802F03DFA10BD300DFF1F3409FF1F1E
:101E40003867FF1F7102000070B5244D2B68002B0E
:101E500028D002F03DF82B68D8402B680400002BF6
:101E600027D002F08DF82B68D8401D4B1D4A997879
:101E7000A1239B004B431268D118D25C91239B0095
:101E8000002A20D0CA580132CA50174B17491B6884
:101E90000868834214D3D23B181A012A1AD0144B73
:101EA000186070BD02F014F8124B196802F0D8F9EE
:101EB000D3E702F065F80F4B196802F0D1F9D4E7C7
:101EC0000D495B18E8E7CA500C4B1B68DB68E41847
:101ED000201AE4E7F530FF30E1E7C0461C08FF1F99
:101EE000300DFF1F3409FF1F9C09FF1F3C67FF1FB8
:101EF000A009FF1F1808FF1F2DFF3F004467FF1FA9
:101F000070B504000D00282916D10300A433C2883F
:101F10001B889B1A0B4A9BB293420DD906006A3666
:101F200005223100653001F0BBFF002804D13100EB
:101F3000200002F0B5F970BD2900200002F070F811
:101F4000F9E7C046FE7F0000F8B50400012002F06A
:101F500047F802F005F8174A1749106009680300AE
:101F60001648174E01601748776805680020AF4291
:101F700001D27068281A144D091928601348C162EB
:101F8000A421446A49032143416211490978002987
:101F900005D010490978022902D10F3B1360F8BD22
:101FA000012901D1083BF9E7032901D1053BF5E7F8
:101FB000033BF3E7E408FF1F28F00040340AFF1F4B
:101FC00028100040180AFF1F1C0AFF1F00F00040E5
:101FD0001C09FF1F4A0AFF1F70B580241025E40565
:101FE000A3682B43A36001F063FFA368AB43A36026
:101FF00070BD0000F7B5160080221C001023D2052A
:102000000191916805000B43936000225A4BD73031
:102010001A6002F0DDF89D232A002F009B00EB5888
:10202000CA3201210092FC37002B01D00021009A16
:10203000386802F045F92900009BCB311A784F4BE4
:10204000D3351A604B780A781B0213438A7812043E
:102050001A43CB781B061343494A1BBA13604B79CA
:102060000A791B0213438A7912041A43CB7931008F
:102070001B061343434A1BBA13606B782A781B0272
:102080001343AA7812041A43EB781B0613433E4A03
:102090001BBA1360019A330213433C4A13603C4B52
:1020A00022001B1B9C4603293DDCB3089A00130049
:1020B0005142B21A032A46D1354AE018511A8278A1
:1020C0004078120400020243E05C043302430A60D9
:1020D0000022FF2B4BDDF0222E4B12011A600F2243
:1020E0002D4B1A602D4A1368002BFCD00023224A86
:1020F00027491360091B321D0B191B68043A180A83
:1021000023706070180C1B0EA070E3700434002A5A
:10211000F2DC802210213B68D20501333B609368DA
:102120008B439360F7BD6346D578981893782D0656
:102130001B042B43157804392B43557804322D02A8
:102140002B430360AFE7022A0AD1114AE05C511A1F
:10215000E2185278120202430A6004339BB2B7E7D6
:10216000012AB5D10A4A521AE15C1160F5E7084923
:1021700059180A600433ACE7000004403C000440F6
:102180003800044034000440300004400C00044097
:102190000001044004000440100004401400044006
:1021A000F7B5150080221C001023D205009191681C
:1021B00007000B4393600023654AD730136002F099
:1021C00007F89D233E009B00F9583B00CA363200B9
:1021D000FC33002900D07FE0586802F071F8390024
:1021E00032785C4BCB311A604B780A781B02134370
:1021F0008A78AC4612041A43CB78281D1B06134379
:10220000554A1BBA13604B790A791B0213438A792A
:1022100012041A43CB791B061343504A1BBA1360AE
:102220004B7A0A7A1B0213438A7A12041A43CB7A36
:1022300021001B0613434A4A1BBA1360009A2B0263
:102240001343484A13602200474B1B1B0093009B1B
:10225000CE785B1801938B7836061B0433430E78D7
:10226000043833434E78043136023343019E3360E1
:102270000328ECDC0321A808431C9B0029408000B4
:1022800003292BD13849E5185E18A9786D78E35CED
:1022900009042D022943194331600300083300214A
:1022A000FF2B2DDD314B324919600F21314B196065
:1022B000012327490B60304B19680029FCD0062107
:1022C0001B680B40042B20D080220020D20593688D
:1022D0000A318B439360FEBD01217DE7022908D1BD
:1022E00021495D18E1184978E35C09021943296026
:1022F000D3E70129D3D11C495918E35C0B60CCE723
:102300001948181801600433CAE7002310490B600C
:102310006346002B0CDC3B00FC335A681021013271
:102320005A608022D205936801208B439360D2E7E4
:10233000009B9B181B68190A13705170190C1B0E17
:10234000D37004235B4291709C440432E0E7C046A2
:10235000000004403C0004403800044034000440C5
:10236000300004400C00044000010440040004401C
:10237000080F0000100004401400044070B5061E51
:1023800019D00222614B9B799343012B13D1604BEF
:102390001A78FF2A0FD15A78FF2A0CD19A78FF2A8F
:1023A00009D1DA78FF2A06D11A79FF2A03D15B799D
:1023B000FF2B00D1A7E0574B0C201A78012A08D038
:1023C0000022554D1A702B781A00093A042A01D8B8
:1023D000212070BD5A1F012AFAD94C4CA07B042839
:1023E00000D990E0A279032A00D98CE0821E012A4C
:1023F00003D862881F2A00D885E0002E61D0012E04
:1024000000D080E0A288012AE2D0002B0AD1013856
:10241000032803D801F0EEFC151D19151F202E709E
:1024200001F00EFF2B785A1E032A16D800253B4BCD
:102430001D602823237501F02BFEA8422ED0A58015
:10244000C6E7022320202B70EAE7042322202B700A
:10245000E6E7032321202B70E2E7073B012BB7D8E7
:102460002F4B1B68DB6A9B06B2D52E4B1A78002ACD
:10247000AED1A27B911E012901D9002AA8D1022246
:1024800080211A702823284D89012878237501F0AE
:10249000BFFE80212878890101F042FD0123A3803D
:1024A000224B1B78002B0AD0FA228021204B92006D
:1024B0001B8809025A431C4B187801F021FD0020AB
:1024C00087E701F07DFD2B78A680073B012B06D91D
:1024D00018482E7001F0CCFC1E2001F0B1FE114B0B
:1024E000114C1A78002A06D0802100222078890118
:1024F0001A7001F08DFE01F0F3FC802120780902B2
:1025000001F086FEDBE7122063E7C046A60BFF1F43
:102510006B09FF1F1A09FF1F1C09FF1F4809FF1F36
:102520004467FF1F2309FF1F1B09FF1F2109FF1F0E
:102530002C09FF1F0010004010B5002901D001F048
:10254000B7FD10BDF7B5604B01919978A1239B00B1
:102550004B435E4A060014681022E418D6235B0041
:10256000E0583623FF33E35C00279343222B41D10D
:10257000574B0F3A1A600760012501F0C1FD019B1E
:102580001880E8235B00E35C002B01D0B34258DDE8
:102590000023504FFB70AD33FF33E3581A68002A15
:1025A00003D09B88DB439B071DD03823FF33E35CBC
:1025B000002B18D09B235B00E35C002B13D1D1339D
:1025C000FF33E35CB3420EDAA4235B00E15AE01868
:1025D000090A023101F02CFC23000122FE33013EE6
:1025E00001351A87FA70E8235B00E35C002B2AD0E0
:1025F000A8B2FEBD03683D00002BBED08188043028
:10260000090A023101F014FCD6235B00E3581F6075
:10261000B2E72300B133BA00FF33985801378188FD
:102620000430090A023101F003FCE8235B00E35C9B
:10263000BB42EEDCE822F61AED1800235200A35448
:10264000A6E70027F1E7200001F062FC00281FD078
:10265000002E1DDD7319882647190193B60020004E
:1026600001F01EFD5A308000201840680135818835
:102670000430090A023101F0DBFB200001F0D8FD33
:10268000A3590133A351BD4202D0019B9D42E6D123
:10269000114BE35C002BABD095239B00E35C002B3C
:1026A000A6D00E4BE15A0029A2D00D4AA35C994254
:1026B00002D90133A3549BE700231A212000A3541D
:1026C00001F0AEFD94E7C046300DFF1F3409FF1F37
:1026D00000140340E010FF1F5A02000072020000C5
:1026E0005E020000F8B51D4B1D4F1A78002A10D16C
:1026F000BA7B002A02D101321A7003E0032AFAD011
:10270000022AF8D001F0C4FC00220120154B1A70F7
:10271000F8BD154B154D1C68154B9E7801232B7089
:102720002878C0B200F0C2FDBB7B002B0BD101F0BA
:1027300037FDA1239B007343E41883239B00E41817
:1027400023782B70E4E7032B02D101F0E1FDF0E7E1
:102750000020022BDCD101F08BFDEAE71C09FF1FF2
:10276000A60BFF1F2309FF1F3409FF1F490AFF1F84
:10277000300DFF1FF0B587B00EAD2F780FAD2D785F
:102780000593AC46634614000E4D0CAA12782E78C1
:1027900003930D9B009201932200059B029701F089
:1027A00037FC2E70012C01D0042C08D18022064960
:1027B0008B889343054A1278D20113438B8007B06C
:1027C000F0BDC0461C09FF1F6C11FF1F7809FF1FD9
:1027D00070B5050001F0A4FD041E32D1A1239B00B9
:1027E0006B43254A1068C01803008F331B78002BF9
:1027F00004D003008B331B78182B3BD098235B004D
:10280000C35C012B36D0FE231C4AFF33C35C825CC1
:102810001A40FF235B00C35C1340194A815C02002D
:102820000D00FE321D40194204D0FA23FF33C15C73
:102830008D4208D10023D38518219386138601F099
:10284000EFFC200070BD02231D4201D0994207D148
:1028500004260123354203D03300B14200D1033BAB
:102860009621490043542E21FF314354038F0733EF
:102870009BB2E1E73A24E4E73409FF1F01020000BC
:1028800002020000F0B585B01D000AAB1B880400F1
:1028900016000191039301F043FD071E6CD1A123A3
:1028A0009B006343394A1468E4182300FF33029302
:1028B0005B7B002B06D120000E3008223449FF300C
:1028C00001F0DEFA029BDA7B09231A425BD0230077
:1028D0008F331B78002B04D023008B331B78162BEF
:1028E0004FD098235B00E35C012B4AD082239B00EE
:1028F000E35C012B45D0274BE35C012B41D0019BCE
:10290000002B01D1AE423ED133002B43072B3AD8E6
:10291000012233001340164205D102231E4202D188
:10292000DE401640B30001212A000A400D4205D1C5
:102930000222154202D1D5400D40AA00019900297A
:1029400006D001291BD01A00022901D001231A0048
:10295000FE21019849006054FE21FF316354FF239A
:102960005B00E254039A0633E252E839103BE0542C
:10297000FF39200001F054FC380005B0F0BD130011
:10298000E6E73A27F8E71127F6E7C0463409FF1FC4
:10299000490EFF1F070200000B001B3B70B504002F
:1029A0003020E02B0DD81300E025493BFF3B9BB2C4
:1029B000ED00AB4205D8034B200019825A8201F08A
:1029C00067FA70BD8410FF1F10B501F0B9FA054B0E
:1029D00000205B68052B04D9034A5268D20200D458
:1029E000980810BD00100040FCE100E070B501F057
:1029F000E7FA0D4B1B68FC33DC691D6AFFF7E4FF47
:102A00006419844204D2094B01241B68002B07D0AF
:102A100004220024064B1A70064A9369013393611D
:102A200001F05EFA200070BD4467FF1F9809FF1F88
:102A30002309FF1FFC0FFF1F70B50C4D2B68FC33E3
:102A40005C6A01F0BDFAFFF7BFFF2B680025FC337D
:102A50009B6AE318834204D2054B1B68AB4200D14A
:102A6000051B01F03DFA280070BDC0464467FF1FFA
:102A70009809FF1FD722044B92009B5810B5002BDA
:102A800000D0984710BDC0460000FF1FF0B587B0CA
:102A900001F03AF9FFF7EEFFCA4BCB4C04931B78D9
:102AA000022B45D1C94B1B68186A01F099FAC84B33
:102AB000C84A1A60C84BC94A1A60A022C84B5200C3
:102AC0001A60049B187801F03BFBC649C64801F028
:102AD0005FFBC649C64801F05BFB1022C54BFF20D7
:102AE0001A60802252031A60802292031A608022A8
:102AF00012041A6001F014FB012001F051FAFA20CF
:102B0000400001F015FA582001F03AFBBA4801F0F4
:102B10009FFA012001F06CFB072001F031FC2268D4
:102B2000B64B1A4084235B001343236007B0F0BD0B
:102B300001F08EF9B24E0290322001F051FA336862
:102B40001B0629D43C2001F04BFA0F2001F048FA73
:102B50009C4B1B78012B00D11EE180223368A94DCC
:102B6000134200D0A7E02B68032013432B6001F031
:102B700037FA01F06DF9029B0299C31A5A1E81427D
:102B800000D81A00A04B1A60904B19681E235343BB
:102B90009E4A9B18CB618AE701F05AF980239C4A30
:102BA000DB02116803900B4313602268934B994F2B
:102BB0001A40282313432360032001F011FA032055
:102BC0003D6801F00DFA3B680320DB03DB0B00934B
:102BD00001F006FA3B68ED03DB03ED0BDB0B8E4ADD
:102BE0000193AB18C22B30D8009B9B18C22B2CD85A
:102BF000019B9B18C22B28D8009B2A009D4200D223
:102C00001A00009B9D4200D91D00019B934200D2F7
:102C10001300019A954200D915005B1B122B14D8A2
:102C20000C22336814209343336033687B4A13408B
:102C3000336001F0D5F908213B682268DB038A4341
:102C40002260774ADB0B13607FE7032001F0C8F9AD
:102C50003B68DB03DB0B059301F0FAF8039B039958
:102C6000C21A531E814200D813006E4A93421BD9E8
:102C7000FF23356869492D0A1D4032686B1C1B060D
:102C80000A401B0C134333600C23326800209A4324
:102C9000083B1343336001F053FB6348634BA84088
:102CA000984206DCFEF74EFE019B009D0093059BBB
:102CB00095E75F48F6E700235E4F554A3B60802367
:102CC0001168DB020B43136080222B68032013433F
:102CD0002B6001F085F93B68052601333B608023BA
:102CE0002A685B0213432B602268444B03201A407E
:102CF000514B1343236001F073F90821454B1A68C7
:102D00002368D2038B432360454B023900931B6831
:102D1000D20B4B439A420CD89B1A3B2B0BD82368FF
:102D200046490B4023602B680B402B60444B1A60D4
:102D30001FE7D31AF1E7013EF6B2002ED4D1236883
:102D40003E4A134023602B6813402B603B68042BE2
:102D500007D9BFF34F8F3B4B3B4ADA60BFF34F8F2E
:102D6000FEE780222B68032093432B6001F038F9A3
:102D70002268224B03201A4028231343236001F0CA
:102D80002FF9244B009A1B68DB03DB0B136008222E
:102D900023689343236097E707222C4D2B68134049
:102DA000012B02D1002001F0CBF9AB68284A0220A8
:102DB0001340AB6001F014F98023AA685B00134351
:102DC000AB60D6E64A0AFF1F5CF000404467FF1F75
:102DD000000003400180063DBC00034034080000B1
:102DE000A40003407102000014100040FFFF3F00E8
:102DF0002810004000E100E03075000000FEFEFFFA
:102E0000C4F0004044F000402C67FF1F7206000031
:102E100040F0004064F0004091FCFFFFFF00FFFF26
:102E20003467FF1FE30C0000E88000005F361E00DF
:102E300060361E00C045FF1F28000100FFFFFEFF97
:102E40003067FF1F00ED00E00400FA053CF0004091
:102E5000FFFEFFFF694E336888331B6883F30888E1
:102E600001F076F900F0C4FB654B664A1B6893429B
:102E700007D0002001F064FA0221634A13688B43F3
:102E80001360FFF703FE614B614C1878C0B201F08C
:102E90003FF90023A3600233A3605E4B012023604F
:102EA00001F09EF80323A36000F0D2FF040001F0BC
:102EB00047F8050000F0CCFF574B186001F0E0F830
:102EC000564B1968621A531EA14200D21300802289
:102ED000D203934201D39B029B0A3268D16AC9078D
:102EE00000D478E04E491C0C09689BB24C4359430E
:102EF0002402090A641803274A49FC3293680A68C5
:102F000049489B1A494A4A4E12684A499B18414A05
:102F100034609A183B400193036892089C46019BD9
:102F20000A6063440360042B03D901323B400A600A
:102F300003600B684049E418200001F091F93F4F0D
:102F40003D493B68C3183B602000019301F0F0F855
:102F50003B4C2068081838492060884205D9019BFD
:102F600001333B6001F0E4F8216001F001F8354BDA
:102F70001B78002B0ED000F0E3FF3168324B4A1B68
:102F80001B6812189A4233D2591A4919091A2F4844
:102F900001F0FEF82E4C237A002B0FD000F0D0FF6A
:102FA0003168E3684A1B1218934224D9591A491907
:102FB000091A284801F0ECF800232372264B83F30A
:102FC000088801F0D5F8022001F03AF9002001F05C
:102FD000B7F901F095F9DC0199000234641A59003F
:102FE000641A09214B438033CB40A408E41882E7DC
:102FF000FA218900CBE71949DBE7C0464467FF1F88
:103000000C0AFF1FB641210310000040490AFF1FB0
:1030100014100040C4090000100AFF1F340AFF1FEB
:10302000380AFF1F200AFF1F280AFF1F1C0AFF1F64
:103030002867FF1F240AFF1F710200006008FF1F9E
:103040002C0AFF1F1C09FF1FE408FF1F001000408F
:10305000740BFF1F3C10004000000020DC05000046
:10306000A022054B92009B5810B5002B01D0984729
:1030700010BD01F075F8FBE70000FF1FA122054B12
:1030800092009B5810B5002B01D0984710BD01F05D
:1030900067F8FBE70000FF1FA222054B92009B5838
:1030A00010B5002B01D0984710BD01F059F8FBE78F
:1030B0000000FF1FA322054B92009B5810B5002B68
:1030C00001D0984710BD01F04BF8FBE70000FF1F4F
:1030D000A422054B92009B5810B5002B01D09847B5
:1030E00010BD01F03DF8FBE70000FF1F70B500F0D8
:1030F00027FF514B1860042001F0A2F801F0E8F816
:103100000400C30702D400F0E3FF70BD00224B4B64
:103110001A604B4B1878013804282CD800F06AFE4E
:1031200003231B1F2700200000F06AFF0128ECD0BA
:10313000444C2378042B71D101F0D2F8002806D03A
:1031400001F086F8582001F01BF8022323700320B9
:1031500001F076F8D9E7200000F08AFFE6E72000CA
:1031600000F0BEFFE2E7200001F0E2F8DEE7200019
:1031700001F0BEF8DAE701F08BF80500012808D16C
:10318000314B1B78053B012B03D82000FFF768FF6C
:10319000CEE72C4B1B78022B01D0052B20D1022D22
:1031A00028D12A4B9B7BAB431CD12000FFF766FF45
:1031B000254B18780128BBD16405B9D423492522B1
:1031C0004B7B034205D1233A13405A4253412633E5
:1031D0001A000B7D9342ABD9322000F0E9FFA7E73C
:1031E000022D07D1184B1B78052B11D12000FFF7BA
:1031F00053FFDDE7012D0BD1012B03D12000FFF799
:1032000059FF95E7062B03D12000FFF761FF8FE7F9
:10321000200000F0A5FF022D8AD1C9E7032B04D1BD
:103220000B4B987C01F094F891E7072B8FD1094B59
:10323000987B00F0FDFE8AE79C09FF1F9809FF1F9D
:103240009009FF1F2309FF1F1C09FF1FA60BFF1F6B
:10325000BC0BFF1FD40BFF1FFA210A4B0A4A49007F
:103260001A640A4A5A500A4A04395A50094A08311B
:103270009A64094A5A50094A5C315A50084ADA6637
:103280007047C0460000FF1F7527FF1F392AFF1F28
:10329000ED29FF1F7D23FF1FE526FF1F011EFF1FD6
:1032A000D51DFF1F10B500F08DFD10BD8023F7B5B3
:1032B0009C46264B264F01932649274A274D284CEA
:1032C000284B02281AD1604638600868264E3040E4
:1032D000802636033043086001990978002909D116
:1032E0001660224A2A60224A2260E022196891432D
:1032F000A03A1BE08021C9021160F2E766463E60F9
:103300000F68194E3E408027FF023E430E60019930
:10331000097800290DD1176001280ED1154A2A60BD
:10332000154A2260E02219689143C03A0A431A60A4
:10333000F7BD802189021160EEE7E0210F4A0243C8
:103340002A600F4A22601A688A43F0E74B0AFF1F7F
:10335000E0000340D8000340900003400000034019
:103360005000034040000340FFFFE3FF0280063DA2
:10337000804508220180063D80660822008006986C
:1033800080550822F8B51E4B80261A6800201400CC
:103390003440324232D11A681A4F32431A60012245
:1033A0003B68063093433B6000F01AFE0122164D45
:1033B0002B681E432E603B680A2613433B60802720
:1033C000BF00124B1B683B4211D1013EF6B2FF2EEB
:1033D00009D17E220E4B1C682B68E40B14409343EA
:1033E00023432B6005E0082000F0FAFDE9E7002EFA
:1033F000EFD180222B68600893432B60F8BDC04654
:10340000C4F000405CF0004018F0004068F000405C
:1034100060F0004010B500F06BFE01215820034A17
:1034200000F0A6FFFFF7AEFF10BDC046600AFF1F09
:1034300010B578220021034800F012FE00F088FD4C
:10344000002010BD4C6AFF1F70B5040000F0B8FDED
:1034500000230C200B4A010059438D18515C0029B0
:103460000DD0A14208D1012300246B7000F0E8FDCB
:1034700000F036FD200070BD01330A2BEBD1122481
:10348000F6E7C0464C6AFF1F70B5040000F098FDD7
:10349000002319001D000D4A1078002806D0A04214
:1034A0000CD1557001310C320A29F5D1002B0AD10B
:1034B00000F04EFD00F014FD002070BD5078461E57
:1034C000B0411B18EEE700F0BBFDF3E74C6AFF1FAD
:1034D000F7B504000C20002384460E4D0192674688
:1034E0005F43E85D7E19A04212D000280BD10A4B41
:1034F0009C4662461B7808331370019B70707C55A4
:103500007160B360FEBD01330A2BE8D10320F9E7F7
:103510000720F7E74C6AFF1F486AFF1F8021204BF6
:10352000C9051B6870B58B601E4BC1241A68012346
:10353000FF2013434B611C4BA4001A681B4B002552
:103540001A601B4B1A681B4B1A601B4B1A5982439B
:103550001A51C52292009C588443BF38204398508A
:103560009C58164804408020C00120439850985829
:10357000134C0002000A01439950124B1B78DB08E0
:10358000AB4201DC002070BD2378002B06D0A3687D
:10359000002B00D0984701350C34EEE71220F2E7FB
:1035A0005846FF1F5446FF1FB0F00040446AFF1FFB
:1035B000B4F00040406AFF1F00E100E0FF00FFFFA1
:1035C0004C6AFF1F486AFF1F030010B51F2809D867
:1035D000072200201340072404490A78A24313431A
:1035E0000B7010BD00230620F5E7C046486AFF1F98
:1035F000034A0449136800200B4013607047C0461B
:103600001CF00040FFFFC1FF054B06491B780A680C
:1036100005485B0702401B0B134300200B607047FB
:10362000486AFF1F1CF00040FFFFC1FF70B50C256A
:10363000FFF7EAFF0A4B1C780A4BE4086543ED18D4
:10364000002C01D1200070BD2B78002B06D06B68B8
:10365000002B00D09847013C0C3DF1E71220F2E727
:10366000486AFF1F406AFF1F07B50422074801A9E7
:1036700000F034F9019B013305D18023044ADB04B7
:1036800011680B43136000200EBDC0461C180011CA
:1036900014F0004007B500F093FC80220821D20509
:1036A000936A0191002B01D10739916202210C4AE2
:1036B00011600199481E01900029FAD1033111606F
:1036C000053101910199481E01900029FAD111603C
:1036D000002B02D18022D205936200F001FC07BDCD
:1036E00000C00040F0B505002026184B87B00493B9
:1036F000049B002B03D11124200007B0F0BD002152
:1037000002220B0001910091052000F099FB022399
:103710000F490A681A42FCD10596059C631E059361
:10372000002CFAD10B4A1368002BFCDA0F276F44E8
:103730000121380000F0DCFB3B782B42DCD0052077
:1037400000F04EFC049B013B0493D1E7FFFFFF0711
:1037500090C8004000C80040F0B52D4C89B02378D7
:10376000002B4FD1FEF7CEF802232A4F03903A6880
:103770001A42FCD120230693069B5A1E0692002B68
:10378000FAD1254E3368002BFCDA0120FFF7AAFF9F
:10379000011E02D0112009B0F0BD030003220190E8
:1037A000009005AD9F2000F04BFB0321280000F0A6
:1037B0009FFB02233A681A42FCD120230793079B00
:1037C0005A1E0792002BFAD13368002BFCDA012035
:1037D000FFF788FF0028DDD10398FEF7A7F8AA7845
:1037E0006B7811041B020B4329780B4363601300B1
:1037F000113B0A49052B07D801239340A3600B60B6
:10380000012323700020C6E780231B03F6E7C04690
:103810004046FF1F90C8004000C800409808FF1FA6
:103820001E4B30B55A6818781D4B85B0D3185942D5
:103830004B4101210093002300F012FB194B1A4A5F
:1038400002259A6300221A6510325A658022C4212B
:103850009D65164B1648D202DA6789004258154B0F
:1038600080241A4080231B041343435064234120C7
:103870000393E40500F078F9402000F075F96562E3
:10388000039D6B1E0393002DFAD103236362FFF7A0
:1038900001FFA562FFF760FF05B030BD4C46FF1F7A
:1038A00095FFFEF700C80040050001FF04E100E0BD
:1038B00000E100E0FFFF00FF10B5064B18705960F3
:1038C000FFF7AEFF00211320034AFFF701FE00209F
:1038D00010BDC0464C46FF1F2138FF1FF0B5040045
:1038E00085B003920291FEF70DF8882263035B0B0B
:1038F00052051A438023DB059D6A8023274F0092DF
:10390000BA68002601901B039A420CD9F8232600BE
:103910001B041E401C4206D08022214B52025E62D4
:1039200019680A431A60002D0BD100F049FB0222EE
:103930001C4B1A608023DB055A62013A9A6200F040
:10394000CFFA0023039A934220D1002D0AD100F030
:1039500037FB144B03221D608023DB055A629D62F6
:1039600000F0BEFA8023BA681B039A4208D9002EE1
:1039700006D000220A4B0C495A621A680A401A60A3
:103980000198FDF7D3FF002005B0F0BD009A029921
:10399000D2181278CA540133D4E7C0464046FF1FFC
:1039A00000C8004000C00040FFFFFEFFF0B587B038
:1039B000029103920400FDF7A5FF019000F000FBC7
:1039C000802302250122234EDB0535605D629A6269
:1039D00000F086FA204F3B682B42FCD12023049351
:1039E000049B5A1E0492002BFAD11C4D2B68002B0D
:1039F000FCDA0120FFF776FE002802D0112007B084
:103A0000F0BD2000039A029900F05AFB0223040043
:103A10003A681A42FCD120230593059B5A1E059251
:103A2000002BFAD12B68002BFCDA0120FFF75AFE9D
:103A3000051EE3D100F0C4FA80230322DB053560C4
:103A40005A629D6200F04CFA0198FDF76FFFE0B2F8
:103A5000D5E7C04600C0004090C8004000C8004004
:103A6000F0B5802687B00400FDF74CFFF605B36A79
:103A700002250393029000F0A3FA0123244F3D6036
:103A80007562B36200F02CFA224E33682B42FCD1EF
:103A900020230493049B5A1E0492002BFAD11E4D3E
:103AA0002B68002BFCDA0120FFF71CFE002802D057
:103AB000112007B0F0BD200000F08AFA0223019027
:103AC00032681A42FCD120230593059B5A1E0592A9
:103AD000002BFAD12B68002BFCDA0320FFF702FE43
:103AE000041EE5D100F06CFA80230322DB053C6064
:103AF0005A629C6200F0F4F9039B002B01D1FFF79E
:103B0000C9FD0298FDF712FF6B461879D1E7C04650
:103B100000C0004090C8004000C8004007B5000247
:103B200001910422000A01A9FFF740FF0EBD000029
:103B300073B5050005240B4AA3005B429B18196866
:103B40006B46DE1D300000F023FA022804D13378E2
:103B50002B55013CEFD276BD052CFCD00128FAD1C3
:103B60000230F8E7140900111F2807D8012380222A
:103B70008340D20591680B43936070473F2808D873
:103B80000123802220388340D20551690B435361C1
:103B9000F3E75F28F1D80123802240388340D20523
:103BA000116A0B431362E8E71F2807D8012280211E
:103BB0008240C9058B6893438B6070473F2808D8C3
:103BC0000122802120388240C9054B6993434B6113
:103BD000F3E75F28F1D80122802140388240C905EF
:103BE0000B6A93430B62E8E71F2810D8802302007A
:103BF000DB05153A1968012A06D82022914319607D
:103C000019680A431A60704701228240F6E73F288C
:103C100011D880230200DB05353AD968032A06D87B
:103C200010229143D960D9680A43DA60EBE7012298
:103C300020388240F5E75F28E5D842238022181A11
:103C4000413B8340D205516A99435162516A0B430B
:103C50005362D8E710B50400012813D1A0221849F7
:103C600092050B685B015B0913430B60154B164A09
:103C700019681140154A0A431A60402219680A431C
:103C80001A6010BD0028FCD101000A2000F0B8FA2B
:103C900021000B2000F0B4FAC0220A4B92001968F0
:103CA0000A4340211A601A688A431A60B022044904
:103CB00012060B685B015B0913430B60E1E7C0462A
:103CC00014F000401CF000407F00FEFF80FD01006A
:103CD000FA2110B58900C00300F0C2FA00F080F9A3
:103CE00010BD0000044B054A1A60054B1A60002203
:103CF000044B1A607047C046140AFF1F841E000060
:103D0000380AFF1FC4F000400023034A1360034A2F
:103D10001360034A1360704754F0004040F10040C4
:103D200044F10040002310B5184C8AB00093019371
:103D30002378012B27D06946012000F051FA002892
:103D400017D1009B12490293019B06AA0393114BC2
:103D500002A81B680493104B1B68059300F0A8F899
:103D600010220E4906A800F09BF8002804D1FF237A
:103D7000237000200AB010BD0123094A074902A898
:103D8000237000F095F80120F4E7C0464867FF1F54
:103D900010290011082900110C29001120290011F7
:103DA0004C67FF1F13B501246946012000F018FA83
:103DB000034B00940193FFF7B5FF200016BDC046EA
:103DC000BB0B000010B5FFF79FFFFFF7EBFF0028CC
:103DD00002D0024B984710BDFEE7C046E1A20000AA
:103DE00002B4714649084900095649008E4402BC94
:103DF0007047C04602B4714649084900095C490051
:103E00008E4402BC7047C04603B471464908400066
:103E10004900095A49008E4403BC70470000000065
:103E200001B40248844601BC604700BFA1AF000056
:103E300001B40248844601BC604700BFC1150100BF
:103E400001B40248844601BC604700BF496D0100CF
:103E500001B40248844601BC604700BF156B0100F5
:103E600001B40248844601BC604700BFC56D010033
:103E700001B40248844601BC604700BFC1A50000F0
:103E800001B40248844601BC604700BF810E0000B7
:103E900001B40248844601BC604700BF116E0000B7
:103EA00001B40248844601BC604700BFCD4C01000C
:103EB00001B40248844601BC604700BFDD3F0000FA
:103EC00001B40248844601BC604700BFE579021195
:103ED00001B40248844601BC604700BFE90B010001
:103EE00001B40248844601BC604700BF9DA90000A0
:103EF00001B40248844601BC604700BF3D71010027
:103F000001B40248844601BC604700BF8B520100E7
:103F100001B40248844601BC604700BF71B0000094
:103F200001B40248844601BC604700BF0D52010045
:103F300001B40248844601BC604700BF85120100FD
:103F400001B40248844601BC604700BFC95C01005F
:103F500001B40248844601BC604700BFADAE00001A
:103F600001B40248844601BC604700BFBD5C01004B
:103F700001B40248844601BC604700BFD54401003B
:103F800001B40248844601BC604700BF6D0B0100CC
:103F900001B40248844601BC604700BFB10702116A
:103FA00001B40248844601BC604700BF69110100AA
:103FB00001B40248844601BC604700BFF9ED00002F
:103FC00001B40248844601BC604700BF75A90000E7
:103FD00001B40248844601BC604700BFA96F0100DC
:103FE00001B40248844601BC604700BF018900005B
:103FF00001B40248844601BC604700BFE94C01009F
:1040000001B40248844601BC604700BF013401008E
:1040100001B40248844601BC604700BF9D6A0000AD
:1040200001B40248844601BC604700BF51B800009B
:1040300001B40248844601BC604700BFC1F70000DC
:1040400001B40248844601BC604700BF21A90000BA
:1040500001B40248844601BC604700BF8D110100D5
:1040600001B40248844601BC604700BFB70E00009F
:1040700001B40248844601BC604700BF0934010016
:1040800001B40248844601BC604700BFC16601001C
:1040900001B40248844601BC604700BFA9D80000B3
:1040A00001B40248844601BC604700BFD9B000009B
:1040B00001B40248844601BC604700BFE9D4000057
:1040C00001B40248844601BC604700BF95730100FB
:1040D00001B40248844601BC604700BFDD0A01000C
:1040E00001B40248844601BC604700BF05340100AA
:1040F00001B40248844601BC604700BFED6801007E
:1041000001B40248844601BC604700BFCD0C0100E9
:1041100001B40248844601BC604700BF8914010015
:1041200001B40248844601BC604700BFED6B01004A
:1041300001B40248844601BC604700BF090E00007C
:1041400001B40248844601BC604700BFEDA50000F1
:1041500001B40248844601BC604700BFC9A9000001
:1041600001B40248844601BC604700BFE917010062
:1041700001B40248844601BC604700BF7997000043
:1041800001B40248844601BC604700BF79120100B7
:1041900001B40248844601BC604700BF2D6C010099
:1041A00001B40248844601BC604700BFE9F6000044
:1041B00001B40248844601BC604700BF613701007A
:1041C00001B40248844601BC604700BFF9A6000064
:1041D00001B40248844601BC604700BF8944000026
:1041E00001B40248844601BC604700BFE1AC000056
:1041F00001B40248844601BC604700BFE5120100DB
:1042000001B40248844601BC604700BFD565021175
:1042100001B40248844601BC604700BFB3520100AC
:1042200001B40248844601BC604700BF53B9000096
:1042300001B40248844601BC604700BF59760100C2
:1042400001B40248844601BC604700BF1907010061
:1042500001B40248844601BC604700BF6DF600000F
:1042600001B40248844601BC604700BF090E00004B
:1042700001B40248844601BC604700BF19FA00003F
:1042800001B40248844601BC604700BFE927000032
:1042900001B40248844601BC604700BFDD0C010048
:1042A00001B40248844601BC604700BF85C10000DC
:1042B00001B40248844601BC604700BF8937010051
:1042C00001B40248844601BC604700BF214400009D
:1042D00001B40248844601BC604700BFBD0B010029
:1042E00001B40248844601BC604700BF01D700000A
:1042F00001B40248844601BC604700BFF9350100A3
:1043000001B40248844601BC604700BF85520100E9
:1043100001B40248844601BC604700BF75F8000044
:1043200001B40248844601BC604700BF1130000060
:1043300001B40248844601BC604700BFF535010066
:1043400001B40248844601BC604700BF016C010013
:1043500001B40248844601BC604700BF4DF900002B
:1043600001B40248844601BC604700BF8D82000052
:1043700001B40248844601BC604700BF01670100E8
:1043800001B40248844601BC604700BFF90D01003A
:10439000020000007E82021101000000A8800211CC
:1043A000020000007A82021101000000D043FF1FCA
:1043B00002000000B080021101000000A464FF1F91
:1043C0000200000078820211030000002464FF1F35
:1043D00012000000020000007E82021101000000B5
:1043E000F0800211020000007A8202110100000038
:1043F000ED80021102000000FA80021103000000AB
:104400005E64FF1F020000007A82021101000000BA
:10441000EC80021102000000F8800211030000008D
:104420003564FF1F020000007882021103000000C3
:104430005664FF1F020000007E820211010000008E
:1044400034810211020000007A8202110100000092
:104450000945FF1F02000000468102110100000013
:104460002B810211020000007A820211010000007B
:104470000845FF1F020000004481021101000000F6
:104480007264FF1F020000007A8202110100000026
:104490000745FF1F020000004281021101000000D9
:1044A0001B810211020000007A820211010000004B
:1044B0000645FF1F020000004081021101000000BC
:1044C00016810211020000007A8202110100000030
:1044D0000545FF1F020000003E810211010000009F
:1044E00011810211020000007A8202110100000015
:1044F0000445FF1F020000003C8102110100000082
:104500000C8102110202020202020000B516021121
:10451000B11602117081021190011D0018001800DF
:10452000FFFF070102030405060201060000000068
:10453000000000000000000000000000000000007B
:104540000000000000000000030000000200000066
:104550007E82021101000000F081021102000000C1
:104560007A82021101000000BC45FF1F020000001A
:10457000FA810211010000009E64FF1F020000008A
:104580007882021103000000F866FF1F020000009D
:104590007A82021101000000BC45FF1F02000000EA
:1045A000F881021101000000A064FF1F020000005A
:1045B0007882021103000000F066FF1F1200000065
:1045C00001000000818102110B000500F7000000CE
:1045D000B4000028002800283075A000A000A0002A
:1045E000A00000080008E001F0001000100010001A
:1045F000100010001000500050005000100010007B
:10460000D0070000000000000F0001000500307519
:1046100007001000010081FF00000000FF00000003
:10462000CD370211D535021165330211FFFF0100AC
:10463000FF000000C9610211455F02115D5E0211B9
:10464000000000000000000000000800040000005E
:104650003B0001085902E00188212800FF0000000A
:10466000020000007E82021101000000448302115A
:10467000020000007A82021101000000DD46FF1FE7
:10468000020000007682021101000000046BFF1F8F
:10469000020000007A82021101000000DC46FF1FC8
:1046A000020000007482021101000000DA46FF1FC0
:1046B000020000007A82021101000000D846FF1FAC
:1046C000020000007282021101000000D046FF1FAC
:1046D000180018001D0090010200000302020000F3
:1046E000020000007E8202110100000058830211C6
:1046F000020000007A820211010000002047FF1F23
:1047000002000000708202110000000000000000A2
:10471000020000007882021103000000246BFF1FDA
:0247200020FF78
:040000051FFF184180
:00000001FF
